 Memory

 Timestamp is 54e2a599 (Mon Feb 16 20:21:13 2015)

 Preferred load address is 10000000

 Start         Length     Name                   Class
 0001:00000000 00006b36H .text                   CODE
 0001:00006b40 0000040aH .text$x                 CODE
 0001:00006f50 0000002cH .text$yc                CODE
 0001:00006f80 0000002bH .text$yd                CODE
 0002:00000000 00000124H .idata$5                DATA
 0002:00000130 00000700H .rdata                  DATA
 0002:00000830 0000006cH .rdata$debug            DATA
 0002:0000089c 0000025cH .rdata$r                DATA
 0002:00000b00 00000088H .rdata$sxdata           DATA
 0002:00000b88 0000067cH .xdata$x                DATA
 0002:00001204 00000050H .idata$2                DATA
 0002:00001254 00000014H .idata$3                DATA
 0002:00001268 00000124H .idata$4                DATA
 0002:0000138c 000004f6H .idata$6                DATA
 0002:00001890 00000994H .edata                  DATA
 0003:00000000 00000158H .data                   DATA
 0003:00000158 000024b0H .bss                    DATA
 0004:00000000 0000000cH .CRT$XCU                DATA
 0004:0000000c 00000008H .CRT$XIC                DATA
 0005:00000000 000000a0H .rsrc$01                DATA
 0005:000000a0 00000548H .rsrc$02                DATA

  Address         Publics by Value              Rva+Base       Lib:Object

 0000:00000022       ___safe_se_handler_count   00000022     <absolute>
 0001:00000000       ??0MMThreadLock@@QAE@PAVMMThreadLockObj@@@Z 10001000 f i Memorylib.obj
 0001:00000020       ??1MMThreadLock@@QAE@XZ    10001020 f i Memorylib.obj
 0001:00000070       ?Enter@MMThreadLockObj@@QAEXXZ 10001070 f i Memorylib.obj
 0001:00000080       ?Exit@MMThreadLockObj@@QAEXXZ 10001080 f i Memorylib.obj
 0001:00000090       ?MemAddIgnoreFileLine@@YGXPBDK@Z 10001090 f   Memorylib.obj
 0001:000000a0       ?MemCBAlloc@@YGXP6GXABQAU_HMEMPOOL@@ABUMEMBLOCKINFO@@@Z@Z 100010a0 f   Memorylib.obj
 0001:000000d0       ?MemCRTAlloc@@YGPAXIH@Z    100010d0 f   Memorylib.obj
 0001:00000160       ?MemCRTFree@@YGXPAXH@Z     10001160 f   Memorylib.obj
 0001:000001d0       ?MemConvertAddress@@YG?AW4MEMCONVERTADDRESSRESULT@@JQAD@Z 100011d0 f   Memorylib.obj
 0001:00000200       ?MemPoolAlloc@@YGPAXPAU_HMEMPOOL@@I@Z 10001200 f   Memorylib.obj
 0001:00000290       ?MemPoolCount@@YGIXZ       10001290 f   Memorylib.obj
 0001:000002d0       ?MemPoolCreate@@YGPAU_HMEMPOOL@@PBDI@Z 100012d0 f   Memorylib.obj
 0001:00000370       ?MemPoolDefault@@YGPAU_HMEMPOOL@@XZ 10001370 f   Memorylib.obj
 0001:00000380       ?MemPoolDestroy@@YGXPAU_HMEMPOOL@@@Z 10001380 f   Memorylib.obj
 0001:00000450       ?MemPoolFree@@YGXPAU_HMEMPOOL@@PAX@Z 10001450 f   Memorylib.obj
 0001:000004d0       ?MemPoolList@@YGIQAPAU_HMEMPOOL@@I@Z 100014d0 f   Memorylib.obj
 0001:00000530       ?MemPoolLock@@YGXPAU_HMEMPOOL@@@Z 10001530 f   Memorylib.obj
 0001:000005a0       ?MemPoolName@@YGPBDPAU_HMEMPOOL@@@Z 100015a0 f   Memorylib.obj
 0001:00000620       ?MemPoolSize@@YGXPAU_HMEMPOOL@@AAI1@Z 10001620 f   Memorylib.obj
 0001:000006c0       ?MemPoolSnapshot@@YGPAU_HMEMPOOLSHOT@@PAU_HMEMPOOL@@@Z 100016c0 f   Memorylib.obj
 0001:00000750       ?MemPoolSnapshotDestroy@@YGXPAU_HMEMPOOLSHOT@@@Z 10001750 f   Memorylib.obj
 0001:000007c0       ?MemPoolUnlock@@YGXPAU_HMEMPOOL@@@Z 100017c0 f   Memorylib.obj
 0001:00000830       ?MemPoolValidate@@YGXPAU_HMEMPOOL@@@Z 10001830 f   Memorylib.obj
 0001:000008a0       ?MemPoolWalkDestroy@@YGXPAU_HMEMPOOLWALK@@@Z 100018a0 f   Memorylib.obj
 0001:00000910       ?MemPoolWalkFirst@@YGPAU_HMEMPOOLWALK@@PAU_HMEMPOOLSHOT@@AAUMEMBLOCKINFO@@@Z 10001910 f   Memorylib.obj
 0001:000009b0       ?MemPoolWalkNext@@YG_NPAU_HMEMPOOLWALK@@AAUMEMBLOCKINFO@@@Z 100019b0 f   Memorylib.obj
 0001:00000a50       ?MemRemIgnoreFileLine@@YGXPBDK@Z 10001a50 f   Memorylib.obj
 0001:00000a60       ?MemSize@@YGXAAI0@Z        10001a60 f   Memorylib.obj
 0001:00000b20       ?MemStringAlloc@@YGPAXII@Z 10001b20 f   Memorylib.obj
 0001:00000bb0       ?MemStringFree@@YGXPAX@Z   10001bb0 f   Memorylib.obj
 0001:00000c20       ?MemVMDumpPool@@YGXPBD0@Z  10001c20 f   Memorylib.obj
 0001:00000cf0       ?MemVMMap@@YGHPBD@Z        10001cf0 f   Memorylib.obj
 0001:00000e30       ?MemVMShrink@@YGXXZ        10001e30 f   Memorylib.obj
 0001:00000e40       ?MemWriteLeakFile@@YGXPBD@Z 10001e40 f   Memorylib.obj
 0001:00000e90       ?MemoryManagerInitialize@@YGXXZ 10001e90 f   Memorylib.obj
 0001:00000ed0       ?MemoryManagerShutdown@@YGXXZ 10001ed0 f   Memorylib.obj
 0001:00001040       ?Release@MMThreadLock@@QAEXXZ 10002040 f i Memorylib.obj
 0001:00001060       ??0MemoryPoolObj@@QAE@ABV0@@Z 10002060 f   MemoryPool.obj
 0001:00001090       ??0MemoryPoolObj@@QAE@PBDI@Z 10002090 f   MemoryPool.obj
 0001:000010c0       ??1MemoryPoolObj@@QAE@XZ   100020c0 f   MemoryPool.obj
 0001:00001110       ??4MemoryPoolObj@@QAEAAV0@ABV0@@Z 10002110 f   MemoryPool.obj
 0001:00001180       ?Handle@MemoryPoolObj@@QAEPAU_HMEMPOOL@@XZ 10002180 f i MemoryPool.obj
 0001:00001190       ?Release@MemoryPoolObj@@AAEXXZ 10002190 f   MemoryPool.obj
 0001:000011e0       ??0FSChunks@?A0x79a48f2f@@AAE@I@Z 100021e0 f i MemorySmall.obj
 0001:00001250       ??0FSPool@?A0x79a48f2f@@QAE@I@Z 10002250 f i MemorySmall.obj
 0001:00001280       ??0MemPoolSmall@@QAE@ABV0@@Z 10002280 f   MemorySmall.obj
 0001:000012c0       ??0MemPoolSmall@@QAE@PBD@Z 100022c0 f   MemorySmall.obj
 0001:00001300       ??0SmallInternals@?A0x79a48f2f@@AAE@PBD@Z 10002300 f i MemorySmall.obj
 0001:00001370       ??1FSChunks@?A0x79a48f2f@@AAE@XZ 10002370 f i MemorySmall.obj
 0001:00001380       ??1FSPool@?A0x79a48f2f@@QAE@XZ 10002380 f i MemorySmall.obj
 0001:000013c0       ??1MemPoolSmall@@QAE@XZ    100023c0 f   MemorySmall.obj
 0001:00001440       ??1SmallInternals@?A0x79a48f2f@@AAE@XZ 10002440 f i MemorySmall.obj
 0001:00001530       ??2@YAPAXIPAX@Z            10002530 f i MemorySmall.obj
 0001:00001540       ??3@YAXPAX0@Z              10002540 f i MemorySmall.obj
 0001:00001550       ??4MemPoolSmall@@QAEAAV0@ABV0@@Z 10002550 f   MemorySmall.obj
 0001:000015f0       ??_GFSChunks@?A0x79a48f2f@@AAEPAXI@Z 100025f0 f i MemorySmall.obj
 0001:00001610       ??_GFSPool@?A0x79a48f2f@@QAEPAXI@Z 10002610 f i MemorySmall.obj
 0001:00001640       ??_GSmallInternals@?A0x79a48f2f@@AAEPAXI@Z 10002640 f i MemorySmall.obj
 0001:00001670       ?AddRef@SmallInternals@?A0x79a48f2f@@QAEPAV12@XZ 10002670 f i MemorySmall.obj
 0001:000016a0       ?Alloc@FSChunks@?A0x79a48f2f@@QAEPAXXZ 100026a0 f i MemorySmall.obj
 0001:000016d0       ?Alloc@FSPool@?A0x79a48f2f@@QAEPAXXZ 100026d0 f i MemorySmall.obj
 0001:00001830       ?Alloc@MemPoolSmall@@QAEPAXI@Z 10002830 f   MemorySmall.obj
 0001:00001840       ?Alloc@SmallInternals@?A0x79a48f2f@@QAEPAXI@Z 10002840 f i MemorySmall.obj
 0001:00001900       ?CalcChunkBuffer@FSChunks@?A0x79a48f2f@@AAEIII@Z 10002900 f i MemorySmall.obj
 0001:00001920       ?CalcChunkMax@FSChunks@?A0x79a48f2f@@AAEIII@Z 10002920 f i MemorySmall.obj
 0001:00001940       ?CalcChunkSizeof@FSChunks@?A0x79a48f2f@@AAEII@Z 10002940 f i MemorySmall.obj
 0001:00001950       ?ChunkLink@FSPool@?A0x79a48f2f@@AAEXPAVFSChunks@2@@Z 10002950 f i MemorySmall.obj
 0001:00001980       ?ChunkUnlink@FSPool@?A0x79a48f2f@@AAEXPAVFSChunks@2@@Z 10002980 f i MemorySmall.obj
 0001:000019c0       ?Create@FSChunks@?A0x79a48f2f@@SGPAV12@I@Z 100029c0 f i MemorySmall.obj
 0001:00001a10       ?Create@SmallInternals@?A0x79a48f2f@@SGPAV12@PBD@Z 10002a10 f i MemorySmall.obj
 0001:00001a40       ?Extend@FSChunks@?A0x79a48f2f@@QAEXXZ 10002a40 f i MemorySmall.obj
 0001:00001ae0       ?Free@FSChunks@?A0x79a48f2f@@QAEXPAX@Z 10002ae0 f i MemorySmall.obj
 0001:00001b10       ?Free@FSPool@?A0x79a48f2f@@QAEXPAX@Z 10002b10 f i MemorySmall.obj
 0001:00001bb0       ?Free@MemPoolSmall@@QAEXPAXI@Z 10002bb0 f   MemorySmall.obj
 0001:00001c30       ?Free@SmallInternals@?A0x79a48f2f@@QAEXPAXI@Z 10002c30 f i MemorySmall.obj
 0001:00001cb0       ?GetAllocCount@FSChunks@?A0x79a48f2f@@QBEIXZ 10002cb0 f i MemorySmall.obj
 0001:00001cc0       ?GetAllocCount@FSPool@?A0x79a48f2f@@QBEIXZ 10002cc0 f i MemorySmall.obj
 0001:00001cf0       ?GetAllocSize@FSPool@?A0x79a48f2f@@QBEIXZ 10002cf0 f i MemorySmall.obj
 0001:00001d00       ?IsNotFull@FSChunks@?A0x79a48f2f@@QBE_NXZ 10002d00 f i MemorySmall.obj
 0001:00001d20       ?IsOwner@FSChunks@?A0x79a48f2f@@QBE_NPBX@Z 10002d20 f i MemorySmall.obj
 0001:00001d50       ?LogIt@SmallInternals@?A0x79a48f2f@@AAEXXZ 10002d50 f i MemorySmall.obj
 0001:00001de0       ?MPeekVMMapSmall@@YGIPAUMPeekSmallChunk@@I@Z 10002de0 f   MemorySmall.obj
 0001:00001ed0       ?Release@FSChunks@?A0x79a48f2f@@QAEXXZ 10002ed0 f i MemorySmall.obj
 0001:00001ef0       ?Release@SmallInternals@?A0x79a48f2f@@QAEXXZ 10002ef0 f i MemorySmall.obj
 0001:00001f60       ?Reset@FSChunks@?A0x79a48f2f@@QAEXII@Z 10002f60 f i MemorySmall.obj
 0001:00001fa0       ?Shrink@FSPool@?A0x79a48f2f@@QAEXXZ 10002fa0 f i MemorySmall.obj
 0001:00002020       ?Shrink@MemPoolSmall@@QAEXXZ 10003020 f   MemorySmall.obj
 0001:00002030       ?Shrink@SmallInternals@?A0x79a48f2f@@QAEXXZ 10003030 f i MemorySmall.obj
 0001:000020d0       ?freeOverloaded@@YGXPAX@Z  100030d0 f   mmCReplacement.obj
 0001:000020f0       ?freeString@@YGXPAX@Z      100030f0 f   mmCReplacement.obj
 0001:00002100       ?mallocOverloaded@@YGPAXI@Z 10003100 f   mmCReplacement.obj
 0001:00002120       ?mallocString@@YGPAXII@Z   10003120 f   mmCReplacement.obj
 0001:00002130       ?_mmstrchr@@YGPBDPBDH@Z    10003130 f   mmCRT.obj
 0001:00002160       ?_mmstrncmp@@YGJPBD0K@Z    10003160 f   mmCRT.obj
 0001:000021c0       _DllMain@12                100031c0 f   mmInit.obj
 0001:00002200       ??0?$MPeekArray@K@?A0x85ca0ab9@@QAE@XZ 10003200 f i mmPeek.obj
 0001:00002210       ??0MPeekFile@?A0x85ca0ab9@@QAE@PBD@Z 10003210 f i mmPeek.obj
 0001:00002250       ??1?$MPeekArray@K@?A0x85ca0ab9@@QAE@XZ 10003250 f i mmPeek.obj
 0001:00002280       ??1MPeekFile@?A0x85ca0ab9@@QAE@XZ 10003280 f i mmPeek.obj
 0001:000022a0       ??A?$MPeekArray@K@?A0x85ca0ab9@@QAEAAKI@Z 100032a0 f i mmPeek.obj
 0001:00002ed0       ?MPeekVMMapDump@@YGHPBD@Z  10003ed0 f   mmPeek.obj
 0001:00003190       ?MPeekVMMapHeaps@@YGHPBDPBUMPeekPool@@I@Z 10004190 f   mmPeek.obj
 0001:00003290       ?MPeekVMMapPool@@YGXPBDK@Z 10004290 f   mmPeek.obj
 0001:00003300       ?MPeekVMMapShrink@@YGXXZ   10004300 f   mmPeek.obj
 0001:00003320       ?MPeekVMMapSmalls@@YGHPBDPBUMPeekSmallChunk@@I@Z 10004320 f   mmPeek.obj
 0001:00003430       ?Resize@?$MPeekArray@K@?A0x85ca0ab9@@QAE_NI@Z 10004430 f i mmPeek.obj
 0001:000034b0       ?Size@?$MPeekArray@K@?A0x85ca0ab9@@QBEIXZ 100044b0 f i mmPeek.obj
 0001:000034c0       ?Write@MPeekFile@?A0x85ca0ab9@@QAEXPBD@Z 100044c0 f i mmPeek.obj
 0001:00003510       ?Writef@MPeekFile@?A0x85ca0ab9@@QAAXPBDZZ 10004510 f i mmPeek.obj
 0001:00003590       ?get@MPeekFile@?A0x85ca0ab9@@QAEPAXXZ 10004590 f i mmPeek.obj
 0001:000035a0       ??0MMAllocInfo@@AAE@XZ     100045a0 f   mmPool.obj
 0001:000035c0       ??0MMAllocTrace@@QAE@XZ    100045c0 f   mmPool.obj
 0001:000035d0       ??0MMPool@@AAE@PBDI@Z      100045d0 f   mmPool.obj
 0001:00003640       ??0MMPoolBase@@IAE@PBDK@Z  10004640 f   mmPool.obj
 0001:00003670       ??0MMSnapshot@@AAE@XZ      10004670 f   mmPool.obj
 0001:00003690       ??0MMSnapshotIterator@@AAE@XZ 10004690 f   mmPool.obj
 0001:000036b0       ??1MMAllocInfo@@AAE@XZ     100046b0 f   mmPool.obj
 0001:000036c0       ??1MMAllocTrace@@QAE@XZ    100046c0 f   mmPool.obj
 0001:000036d0       ??1MMPool@@EAE@XZ          100046d0 f   mmPool.obj
 0001:00003770       ??1MMPoolBase@@MAE@XZ      10004770 f   mmPool.obj
 0001:00003780       ??1MMSnapshot@@AAE@XZ      10004780 f   mmPool.obj
 0001:00003790       ??1MMSnapshotIterator@@AAE@XZ 10004790 f   mmPool.obj
 0001:000037a0       ??_GMMAllocInfo@@AAEPAXI@Z 100047a0 f i mmPool.obj
 0001:000037c0       ??_GMMAllocTrace@@QAEPAXI@Z 100047c0 f i mmPool.obj
 0001:000037e0       ??_GMMPool@@EAEPAXI@Z      100047e0 f i mmPool.obj
 0001:000037e0       ??_EMMPool@@EAEPAXI@Z      100047e0 f i mmPool.obj
 0001:00003810       ??_EMMPoolBase@@MAEPAXI@Z  10004810 f i mmPool.obj
 0001:00003810       ??_GMMPoolBase@@MAEPAXI@Z  10004810 f i mmPool.obj
 0001:00003840       ??_GMMSnapshot@@AAEPAXI@Z  10004840 f i mmPool.obj
 0001:00003860       ??_GMMSnapshotIterator@@AAEPAXI@Z 10004860 f i mmPool.obj
 0001:00003880       ?Add@MMAllocInfo@@QAEPBUAllocEntry@1@PAXIW4MEMBLOCKTYPE@@@Z 10004880 f   mmPool.obj
 0001:00003970       ?AddTrace@MMAllocTrace@@QAEIXZ 10004970 f   mmPool.obj
 0001:00003ab0       ?Alloc@MMPool@@UAEPAXIW4MEMBLOCKTYPE@@P6GXABQAU_HMEMPOOL@@ABUMEMBLOCKINFO@@@Z@Z 10004ab0 f   mmPool.obj
 0001:00003b90       ?AllocExist@MMAllocInfo@@QAE_NABUMEMBLOCKINFO@@@Z 10004b90 f   mmPool.obj
 0001:00003c00       ?AllocExist@MMPool@@UAE_NABUMEMBLOCKINFO@@@Z 10004c00 f   mmPool.obj
 0001:00003c20       ?ClassInitialize@MMPool@@SGXXZ 10004c20 f   mmPool.obj
 0001:00003c40       ?ClassShutdown@MMPool@@SGXXZ 10004c40 f   mmPool.obj
 0001:00003ca0       ?Convert@MMSnapshot@@SGPAV1@PAX@Z 10004ca0 f   mmPool.obj
 0001:00003cc0       ?Convert@MMSnapshotIterator@@SGPAV1@PAX@Z 10004cc0 f   mmPool.obj
 0001:00003ce0       ?ConvertTo@MMPool@@SGPAV1@PAX@Z 10004ce0 f   mmPool.obj
 0001:00003d00       ?Create@MMAllocInfo@@SGPAV1@XZ 10004d00 f   mmPool.obj
 0001:00003d90       ?Create@MMAllocTrace@@SGPAV1@XZ 10004d90 f   mmPool.obj
 0001:00003dc0       ?Create@MMPool@@SGPAV1@PBDI@Z 10004dc0 f   mmPool.obj
 0001:00003df0       ?Create@MMSnapshot@@SGPAV1@PBVMMPool@@@Z 10004df0 f   mmPool.obj
 0001:00003e00       ?DeleteBucket@MMAllocInfo@@AAEXAAPAUAllocEntry@1@PAU21@@Z 10004e00 f   mmPool.obj
 0001:00003e30       ?Destroy@MMAllocInfo@@SGXPAV1@@Z 10004e30 f   mmPool.obj
 0001:00003e80       ?Destroy@MMAllocTrace@@SGXPAV1@@Z 10004e80 f   mmPool.obj
 0001:00003ea0       ?Destroy@MMPool@@UAEXXZ    10004ea0 f   mmPool.obj
 0001:00003ec0       ?Destroy@MMSnapshot@@SGXPAV1@@Z 10004ec0 f   mmPool.obj
 0001:00003ee0       ?ExtendHashTable@MMAllocInfo@@AAEXXZ 10004ee0 f   mmPool.obj
 0001:00004160       ?FindFreeSlot@MMAllocInfo@@AAE_NAAPAUAllocEntry@1@IPAU21@0@Z 10005160 f   mmPool.obj
 0001:000041d0       ?Free@MMPool@@UAEXPAXW4MEMFREETYPE@@@Z 100051d0 f   mmPool.obj
 0001:00004200       ?Get@MMSnapshotIterator@@QBEABUMEMBLOCKINFO@@XZ 10005200 f   mmPool.obj
 0001:00004220       ?GetAlloc@MMPool@@UBEIXZ   10005220 f   mmPool.obj
 0001:00004230       ?GetAllocMax@MMPool@@UBEIXZ 10005230 f   mmPool.obj
 0001:00004240       ?GetAt@MMSnapshot@@QBEABUMEMBLOCKINFO@@I@Z 10005240 f   mmPool.obj
 0001:00004260       ?GetHandle@MMPool@@QBEKXZ  10005260 f   mmPool.obj
 0001:00004270       ?GetMemorySize@MMPool@@UBEIXZ 10005270 f   mmPool.obj
 0001:00004280       ?GetMemorySizeMax@MMPool@@UBEIXZ 10005280 f   mmPool.obj
 0001:00004290       ?GetName@MMPoolBase@@QBEPBDXZ 10005290 f   mmPool.obj
 0001:000042a0       ?GetQty@MMSnapshot@@QBEIXZ 100052a0 f i mmPool.obj
 0001:000042b0       ?GoNext@MMSnapshotIterator@@QAE_NXZ 100052b0 f   mmPool.obj
 0001:000042d0       ?IterCreate@MMSnapshot@@SGPAVMMSnapshotIterator@@PAV1@@Z 100052d0 f   mmPool.obj
 0001:00004330       ?IterDestroy@MMSnapshot@@SGXPAVMMSnapshotIterator@@@Z 10005330 f   mmPool.obj
 0001:00004350       ?Lock@MMPool@@UAEXXZ       10005350 f   mmPool.obj
 0001:00004360       ?MMPoolCheckFree@@YGXW4MEMBLOCKTYPE@@W4MEMFREETYPE@@@Z 10005360 f   mmPool.obj
 0001:00004370       ?MMPoolCheckLeaks@@YGXPBDI@Z 10005370 f   mmPool.obj
 0001:000043b0       ?MMPoolFill@@YGXPAXI@Z     100053b0 f   mmPool.obj
 0001:000043c0       ?MemorySize@MMAllocInfo@@QBEIXZ 100053c0 f   mmPool.obj
 0001:000043d0       ?MemorySizeMax@MMAllocInfo@@QBEIXZ 100053d0 f   mmPool.obj
 0001:000043e0       ?NewBucket@MMAllocInfo@@AAEPAUAllocEntry@1@AAPAU21@@Z 100053e0 f   mmPool.obj
 0001:00004410       ?Rmv@MMAllocInfo@@QAEXPAXW4MEMFREETYPE@@@Z 10005410 f   mmPool.obj
 0001:000044e0       ?Size@MMAllocInfo@@QBEIXZ  100054e0 f   mmPool.obj
 0001:000044f0       ?Size@MMAllocTrace@@QBEIXZ 100054f0 f   mmPool.obj
 0001:00004500       ?Unlock@MMPool@@UAEXXZ     10005500 f   mmPool.obj
 0001:00004510       ?Validate@MMPool@@UAEXXZ   10005510 f   mmPool.obj
 0001:00004580       ??0Internals@MMPoolVM@@AAE@XZ 10005580 f   mmPoolVM.obj
 0001:000045d0       ??0MMPoolVM@@AAE@PBD@Z     100055d0 f   mmPoolVM.obj
 0001:00004610       ??1Internals@MMPoolVM@@AAE@XZ 10005610 f   mmPoolVM.obj
 0001:00004660       ??1MMPoolVM@@EAE@XZ        10005660 f   mmPoolVM.obj
 0001:00004670       ??_GInternals@MMPoolVM@@AAEPAXI@Z 10005670 f i mmPoolVM.obj
 0001:000046a0       ??_EMMPoolVM@@EAEPAXI@Z    100056a0 f i mmPoolVM.obj
 0001:000046a0       ??_GMMPoolVM@@EAEPAXI@Z    100056a0 f i mmPoolVM.obj
 0001:000046d0       ?Alloc@Internals@MMPoolVM@@QAEPAXIW4MEMBLOCKTYPE@@P6GXABQAU_HMEMPOOL@@ABUMEMBLOCKINFO@@@Z@Z 100056d0 f   mmPoolVM.obj
 0001:00004780       ?Alloc@MMPoolVM@@UAEPAXIW4MEMBLOCKTYPE@@P6GXABQAU_HMEMPOOL@@ABUMEMBLOCKINFO@@@Z@Z 10005780 f   mmPoolVM.obj
 0001:000047a0       ?AllocExist@MMPoolVM@@UAE_NABUMEMBLOCKINFO@@@Z 100057a0 f   mmPoolVM.obj
 0001:000047b0       ?ClassInitialize@MMPoolVM@@SGXXZ 100057b0 f   mmPoolVM.obj
 0001:00004820       ?ClassShutdown@MMPoolVM@@SGXXZ 10005820 f   mmPoolVM.obj
 0001:00004860       ?ConvertTo@MMPoolVM@@SGPAV1@PAX@Z 10005860 f   mmPoolVM.obj
 0001:00004880       ?Create@MMPoolVM@@SGPAV1@PBDI@Z 10005880 f   mmPoolVM.obj
 0001:00004910       ?Destroy@MMPoolVM@@UAEXXZ  10005910 f   mmPoolVM.obj
 0001:00004930       ?Free@Internals@MMPoolVM@@QAEXPAXW4MEMFREETYPE@@@Z 10005930 f   mmPoolVM.obj
 0001:000049b0       ?Free@MMPoolVM@@UAEXPAXW4MEMFREETYPE@@@Z 100059b0 f   mmPoolVM.obj
 0001:000049d0       ?GetAlloc@MMPoolVM@@UBEIXZ 100059d0 f   mmPoolVM.obj
 0001:000049e0       ?GetAllocMax@MMPoolVM@@UBEIXZ 100059e0 f   mmPoolVM.obj
 0001:000049f0       ?GetMemorySize@MMPoolVM@@UBEIXZ 100059f0 f   mmPoolVM.obj
 0001:00004a00       ?GetMemorySizeMax@MMPoolVM@@UBEIXZ 10005a00 f   mmPoolVM.obj
 0001:00004a10       ?GetOType@Internals@MMPoolVM@@AAEXAAPAUHeader@12@PAX@Z 10005a10 f   mmPoolVM.obj
 0001:00004a40       ?GetUType@Internals@MMPoolVM@@AAEXAAPAUHeader@12@PAX@Z 10005a40 f   mmPoolVM.obj
 0001:00004a60       ?LargeAlloc@Internals@MMPoolVM@@AAEPAXIW4MEMBLOCKTYPE@@@Z 10005a60 f   mmPoolVM.obj
 0001:00004b40       ?LargeFree@Internals@MMPoolVM@@AAEXPAXPAUHeader@12@W4MEMFREETYPE@@@Z 10005b40 f   mmPoolVM.obj
 0001:00004b70       ?LargeOLock@Internals@MMPoolVM@@AAEXPAUHeaderLarge@12@PAX@Z 10005b70 f   mmPoolVM.obj
 0001:00004ba0       ?LargeORaw@Internals@MMPoolVM@@AAEIIAAPAUHeaderLarge@12@AAPAX@Z 10005ba0 f   mmPoolVM.obj
 0001:00004bf0       ?LargeORel@Internals@MMPoolVM@@AAEXPAXPAUHeaderLarge@12@@Z 10005bf0 f   mmPoolVM.obj
 0001:00004c10       ?LargeULock@Internals@MMPoolVM@@AAEXPAUHeaderLarge@12@PAX@Z 10005c10 f   mmPoolVM.obj
 0001:00004c40       ?LargeURaw@Internals@MMPoolVM@@AAEIIAAPAUHeaderLarge@12@AAPAX@Z 10005c40 f   mmPoolVM.obj
 0001:00004c90       ?LargeURel@Internals@MMPoolVM@@AAEXPAXPAUHeaderLarge@12@@Z 10005c90 f   mmPoolVM.obj
 0001:00004cb0       ?Lock@MMPoolVM@@UAEXXZ     10005cb0 f   mmPoolVM.obj
 0001:00004cc0       ?SmallAlloc@Internals@MMPoolVM@@AAEPAXIW4MEMBLOCKTYPE@@@Z 10005cc0 f   mmPoolVM.obj
 0001:00004e20       ?SmallFree@Internals@MMPoolVM@@AAEXPAXPAUHeader@12@W4MEMFREETYPE@@@Z 10005e20 f   mmPoolVM.obj
 0001:00004eb0       ?SmallNewRegion@Internals@MMPoolVM@@AAEXXZ 10005eb0 f   mmPoolVM.obj
 0001:00005010       ?SmallOLock@Internals@MMPoolVM@@AAEXPAUHeaderSmallInUse@12@PAX@Z 10006010 f   mmPoolVM.obj
 0001:00005040       ?SmallORaw@Internals@MMPoolVM@@AAEXPAUHeaderSmallFree@12@IAAPAUHeaderSmallInUse@12@AAPAX@Z 10006040 f   mmPoolVM.obj
 0001:00005080       ?SmallORel@Internals@MMPoolVM@@AAEXAAPAUHeaderSmallFree@12@PAXPAUHeaderSmallInUse@12@@Z 10006080 f   mmPoolVM.obj
 0001:00005090       ?SmallULock@Internals@MMPoolVM@@AAEXPAUHeaderSmallInUse@12@PAX@Z 10006090 f   mmPoolVM.obj
 0001:000050c0       ?SmallURaw@Internals@MMPoolVM@@AAEXPAUHeaderSmallFree@12@IAAPAUHeaderSmallInUse@12@AAPAX@Z 100060c0 f   mmPoolVM.obj
 0001:00005100       ?SmallURel@Internals@MMPoolVM@@AAEXAAPAUHeaderSmallFree@12@PAXPAUHeaderSmallInUse@12@@Z 10006100 f   mmPoolVM.obj
 0001:00005130       ?Unlock@MMPoolVM@@UAEXXZ   10006130 f   mmPoolVM.obj
 0001:00005140       ?Validate@MMPoolVM@@UAEXXZ 10006140 f   mmPoolVM.obj
 0001:00005150       ?mmStackTraceFast@@YG_NPAJJJ@Z 10006150 f   mmStackTrace.obj
 0001:00005190       ??0MMThreadLockObj@@QAE@XZ 10006190 f   mmThreadLock.obj
 0001:000051a0       ??1MMThreadLockObj@@QAE@XZ 100061a0 f   mmThreadLock.obj
 0001:000051b0       ??_GMMThreadLockObj@@QAEPAXI@Z 100061b0 f i mmThreadLock.obj
 0001:000051e0       ?GlobalLockInit@@YGXXZ     100061e0 f   mmThreadLock.obj
 0001:00005200       ?GlobalLockShutdown@@YGXXZ 10006200 f   mmThreadLock.obj
 0001:00005210       ?mmFormatAllocation@@YGPBDABQAU_HMEMPOOL@@ABUMEMBLOCKINFO@@I@Z 10006210 f   mmWriteHeap.obj
 0001:00005220       ?mmWriteHeap@@YGXPBDK@Z    10006220 f   mmWriteHeap.obj
 0001:00005230       ?mmWritePoolAppend@@YGXABQAU_HMEMPOOL@@PBDK@Z 10006230 f   mmWriteHeap.obj
 0001:00005240       ?VMQuery@@YGHPAXPBXPAUVMQUERY@@@Z 10006240 f   VMQuery.obj
 0001:000054c0       ??$_Allocate@D@std@@YGPADIPAD@Z 100064c0 f i mmgr.obj
 0001:000054f0       ??$addressof@D@std@@YGPADAAD@Z 100064f0 f i mmgr.obj
 0001:00005500       ??$construct@PADAAPAD@?$_Wrap_alloc@V?$allocator@D@std@@@std@@QAEXPAPADAAPAD@Z 10006500 f i mmgr.obj
 0001:00005520       ??$construct@PADAAPAD@?$allocator@D@std@@QAEXPAPADAAPAD@Z 10006520 f i mmgr.obj
 0001:00005540       ??$construct@PADAAPAD@?$allocator_traits@V?$allocator@D@std@@@std@@SGXAAV?$allocator@D@1@PAPADAAPAD@Z 10006540 f i mmgr.obj
 0001:00005560       ??$destroy@PAD@?$_Wrap_alloc@V?$allocator@D@std@@@std@@QAEXPAPAD@Z 10006560 f i mmgr.obj
 0001:00005570       ??$destroy@PAD@?$allocator@D@std@@QAEXPAPAD@Z 10006570 f i mmgr.obj
 0001:00005580       ??$destroy@PAD@?$allocator_traits@V?$allocator@D@std@@@std@@SGXAAV?$allocator@D@1@PAPAD@Z 10006580 f i mmgr.obj
 0001:00005590       ??$forward@AAPAD@std@@YGAAPADAAPAD@Z 10006590 f i mmgr.obj
 0001:000055a0       ??0?$_String_alloc@$0A@U?$_String_base_types@DV?$allocator@D@std@@@std@@@std@@QAE@ABV?$allocator@D@1@@Z 100065a0 f i mmgr.obj
 0001:000055c0       ??0?$_String_val@U?$_Simple_types@D@std@@@std@@QAE@XZ 100065c0 f i mmgr.obj
 0001:000055e0       ??0?$_Wrap_alloc@V?$allocator@D@std@@@std@@QAE@XZ 100065e0 f i mmgr.obj
 0001:000055f0       ??0?$allocator@D@std@@QAE@XZ 100065f0 f i mmgr.obj
 0001:00005600       ??0?$basic_string@DU?$char_traits@D@std@@V?$allocator@D@2@@std@@QAE@PBD@Z 10006600 f i mmgr.obj
 0001:00005650       ??0_Generic_error_category@std@@QAE@XZ 10006650 f i mmgr.obj
 0001:00005660       ??0_Iostream_error_category@std@@QAE@XZ 10006660 f i mmgr.obj
 0001:00005670       ??0_System_error_category@std@@QAE@XZ 10006670 f i mmgr.obj
 0001:00005680       ??0error_category@std@@QAE@XZ 10006680 f i mmgr.obj
 0001:00005690       ??0error_condition@std@@QAE@HABVerror_category@1@@Z 10006690 f i mmgr.obj
 0001:000056b0       ??1?$basic_string@DU?$char_traits@D@std@@V?$allocator@D@2@@std@@QAE@XZ 100066b0 f i mmgr.obj
 0001:000056e0       ??1_Generic_error_category@std@@UAE@XZ 100066e0 f i mmgr.obj
 0001:000056f0       ??1_Iostream_error_category@std@@UAE@XZ 100066f0 f i mmgr.obj
 0001:00005700       ??1_System_error_category@std@@UAE@XZ 10006700 f i mmgr.obj
 0001:00005710       ??1error_category@std@@UAE@XZ 10006710 f i mmgr.obj
 0001:00005720       ??8error_category@std@@QBE_NABV01@@Z 10006720 f i mmgr.obj
 0001:00005730       ??8error_condition@std@@QBE_NABV01@@Z 10006730 f i mmgr.obj
 0001:00005750       ??_G_Generic_error_category@std@@UAEPAXI@Z 10006750 f i mmgr.obj
 0001:00005750       ??_E_Generic_error_category@std@@UAEPAXI@Z 10006750 f i mmgr.obj
 0001:00005780       ??_G_Iostream_error_category@std@@UAEPAXI@Z 10006780 f i mmgr.obj
 0001:00005780       ??_E_Iostream_error_category@std@@UAEPAXI@Z 10006780 f i mmgr.obj
 0001:000057b0       ??_E_System_error_category@std@@UAEPAXI@Z 100067b0 f i mmgr.obj
 0001:000057b0       ??_G_System_error_category@std@@UAEPAXI@Z 100067b0 f i mmgr.obj
 0001:000057e0       ??_Gerror_category@std@@UAEPAXI@Z 100067e0 f i mmgr.obj
 0001:000057e0       ??_Eerror_category@std@@UAEPAXI@Z 100067e0 f i mmgr.obj
 0001:00005810       ?_Copy@?$basic_string@DU?$char_traits@D@std@@V?$allocator@D@2@@std@@QAEXII@Z 10006810 f i mmgr.obj
 0001:00005960       ?_Eos@?$basic_string@DU?$char_traits@D@std@@V?$allocator@D@2@@std@@QAEXI@Z 10006960 f i mmgr.obj
 0001:00005990       ?_Getal@?$_String_alloc@$0A@U?$_String_base_types@DV?$allocator@D@std@@@std@@@std@@QBE?AU?$_Wrap_alloc@V?$allocator@D@std@@@2@XZ 10006990 f i mmgr.obj
 0001:000059a0       ?_Grow@?$basic_string@DU?$char_traits@D@std@@V?$allocator@D@2@@std@@QAE_NI_N@Z 100069a0 f i mmgr.obj
 0001:00005a50       ?_Inside@?$basic_string@DU?$char_traits@D@std@@V?$allocator@D@2@@std@@QAE_NPBD@Z 10006a50 f i mmgr.obj
 0001:00005a90       ?_Myptr@?$_String_val@U?$_Simple_types@D@std@@@std@@QAEPADXZ 10006a90 f i mmgr.obj
 0001:00005aa0       ?_Myptr@?$_String_val@U?$_Simple_types@D@std@@@std@@QBEPBDXZ 10006aa0 f i mmgr.obj
 0001:00005ab0       ?_Tidy@?$basic_string@DU?$char_traits@D@std@@V?$allocator@D@2@@std@@QAEX_NI@Z 10006ab0 f i mmgr.obj
 0001:00005b00       ?_Xlen@?$basic_string@DU?$char_traits@D@std@@V?$allocator@D@2@@std@@QBEXXZ 10006b00 f i mmgr.obj
 0001:00005b10       ?_Xran@?$basic_string@DU?$char_traits@D@std@@V?$allocator@D@2@@std@@QBEXXZ 10006b10 f i mmgr.obj
 0001:00005b20       ?allocate@?$_Wrap_alloc@V?$allocator@D@std@@@std@@QAEPADI@Z 10006b20 f i mmgr.obj
 0001:00005b50       ?allocate@?$allocator@D@std@@QAEPADI@Z 10006b50 f i mmgr.obj
 0001:00005b80       ?assign@?$basic_string@DU?$char_traits@D@std@@V?$allocator@D@2@@std@@QAEAAV12@ABV12@II@Z 10006b80 f i mmgr.obj
 0001:00005ca0       ?assign@?$basic_string@DU?$char_traits@D@std@@V?$allocator@D@2@@std@@QAEAAV12@PBD@Z 10006ca0 f i mmgr.obj
 0001:00005ce0       ?assign@?$basic_string@DU?$char_traits@D@std@@V?$allocator@D@2@@std@@QAEAAV12@PBDI@Z 10006ce0 f i mmgr.obj
 0001:00005de0       ?assign@?$char_traits@D@std@@SAXAADABD@Z 10006de0 f i mmgr.obj
 0001:00005df0       ?category@error_code@std@@QBEABVerror_category@2@XZ 10006df0 f i mmgr.obj
 0001:00005e00       ?category@error_condition@std@@QBEABVerror_category@2@XZ 10006e00 f i mmgr.obj
 0001:00005e10       ?copy@?$char_traits@D@std@@SAPADPADPBDI@Z 10006e10 f i mmgr.obj
 0001:00005e30       ?deallocate@?$_Wrap_alloc@V?$allocator@D@std@@@std@@QAEXPADI@Z 10006e30 f i mmgr.obj
 0001:00005e50       ?deallocate@?$allocator@D@std@@QAEXPADI@Z 10006e50 f i mmgr.obj
 0001:00005e70       ?default_error_condition@_System_error_category@std@@UBE?AVerror_condition@2@H@Z 10006e70 f i mmgr.obj
 0001:00005eb0       ?default_error_condition@error_category@std@@UBE?AVerror_condition@2@H@Z 10006eb0 f i mmgr.obj
 0001:00005ed0       ?equivalent@error_category@std@@UBE_NABVerror_code@2@H@Z 10006ed0 f i mmgr.obj
 0001:00005ef0       ?equivalent@error_category@std@@UBE_NHABVerror_condition@2@@Z 10006ef0 f i mmgr.obj
 0001:00005f30       ?erase@?$basic_string@DU?$char_traits@D@std@@V?$allocator@D@2@@std@@QAEAAV12@I@Z 10006f30 f i mmgr.obj
 0001:00005f70       ?erase@?$basic_string@DU?$char_traits@D@std@@V?$allocator@D@2@@std@@QAEAAV12@II@Z 10006f70 f i mmgr.obj
 0001:00006010       ?generic_category@std@@YGABVerror_category@1@XZ 10007010 f i mmgr.obj
 0001:00006020       ?length@?$char_traits@D@std@@SAIPBD@Z 10007020 f i mmgr.obj
 0001:00006040       ?max_size@?$_Wrap_alloc@V?$allocator@D@std@@@std@@QBEIXZ 10007040 f i mmgr.obj
 0001:00006050       ?max_size@?$allocator@D@std@@QBEIXZ 10007050 f i mmgr.obj
 0001:00006060       ?max_size@?$allocator_traits@V?$allocator@D@std@@@std@@SGIABV?$allocator@D@2@@Z 10007060 f i mmgr.obj
 0001:00006070       ?max_size@?$basic_string@DU?$char_traits@D@std@@V?$allocator@D@2@@std@@QBEIXZ 10007070 f i mmgr.obj
 0001:00006080       ?message@_Generic_error_category@std@@UBE?AV?$basic_string@DU?$char_traits@D@std@@V?$allocator@D@2@@2@H@Z 10007080 f i mmgr.obj
 0001:000060f0       ?message@_Iostream_error_category@std@@UBE?AV?$basic_string@DU?$char_traits@D@std@@V?$allocator@D@2@@2@H@Z 100070f0 f i mmgr.obj
 0001:00006150       ?message@_System_error_category@std@@UBE?AV?$basic_string@DU?$char_traits@D@std@@V?$allocator@D@2@@2@H@Z 10007150 f i mmgr.obj
 0001:000061c0       ?move@?$char_traits@D@std@@SAPADPADPBDI@Z 100071c0 f i mmgr.obj
 0001:000061e0       ?name@_Generic_error_category@std@@UBEPBDXZ 100071e0 f i mmgr.obj
 0001:000061f0       ?name@_Iostream_error_category@std@@UBEPBDXZ 100071f0 f i mmgr.obj
 0001:00006200       ?name@_System_error_category@std@@UBEPBDXZ 10007200 f i mmgr.obj
 0001:00006210       ?size@?$basic_string@DU?$char_traits@D@std@@V?$allocator@D@2@@std@@QBEIXZ 10007210 f i mmgr.obj
 0001:00006220       ?system_category@std@@YGABVerror_category@1@XZ 10007220 f i mmgr.obj
 0001:00006230       ?value@error_code@std@@QBEHXZ 10007230 f i mmgr.obj
 0001:00006240       ?value@error_condition@std@@QBEHXZ 10007240 f i mmgr.obj
 0001:00006244       _DeleteFileA@4             10007244 f   kernel32:KERNEL32.dll
 0001:0000624a       _GetFileAttributesA@4      1000724a f   kernel32:KERNEL32.dll
 0001:00006250       _EnterCriticalSection@4    10007250 f   kernel32:KERNEL32.dll
 0001:00006256       _LeaveCriticalSection@4    10007256 f   kernel32:KERNEL32.dll
 0001:0000625c       _lstrcmpiA@8               1000725c f   kernel32:KERNEL32.dll
 0001:00006262       _lstrcpynA@12              10007262 f   kernel32:KERNEL32.dll
 0001:00006268       _lstrcpyA@8                10007268 f   kernel32:KERNEL32.dll
 0001:0000626e       _lstrlenA@4                1000726e f   kernel32:KERNEL32.dll
 0001:00006274       _OutputDebugStringA@4      10007274 f   kernel32:KERNEL32.dll
 0001:0000627a       _VirtualAlloc@16           1000727a f   kernel32:KERNEL32.dll
 0001:00006280       _VirtualFree@12            10007280 f   kernel32:KERNEL32.dll
 0001:00006286       _DisableThreadLibraryCalls@4 10007286 f   kernel32:KERNEL32.dll
 0001:0000628c       _GetModuleHandleA@4        1000728c f   kernel32:KERNEL32.dll
 0001:00006292       _CreateFileA@28            10007292 f   kernel32:KERNEL32.dll
 0001:00006298       _WriteFile@20              10007298 f   kernel32:KERNEL32.dll
 0001:0000629e       _DebugBreak@0              1000729e f   kernel32:KERNEL32.dll
 0001:000062a4       _CloseHandle@4             100072a4 f   kernel32:KERNEL32.dll
 0001:000062aa       _GetProcessHeap@0          100072aa f   kernel32:KERNEL32.dll
 0001:000062b0       _GetProcessHeaps@8         100072b0 f   kernel32:KERNEL32.dll
 0001:000062b6       _HeapLock@4                100072b6 f   kernel32:KERNEL32.dll
 0001:000062bc       _HeapUnlock@4              100072bc f   kernel32:KERNEL32.dll
 0001:000062c2       _HeapWalk@8                100072c2 f   kernel32:KERNEL32.dll
 0001:000062c8       _GetCurrentProcess@0       100072c8 f   kernel32:KERNEL32.dll
 0001:000062ce       _GetVersionExA@4           100072ce f   kernel32:KERNEL32.dll
 0001:000062d4       _VirtualQuery@12           100072d4 f   kernel32:KERNEL32.dll
 0001:000062da       _GetProcAddress@8          100072da f   kernel32:KERNEL32.dll
 0001:000062e0       _lstrcatA@8                100072e0 f   kernel32:KERNEL32.dll
 0001:000062e6       _LoadLibraryA@4            100072e6 f   kernel32:KERNEL32.dll
 0001:000062ec       _HeapCreate@12             100072ec f   kernel32:KERNEL32.dll
 0001:000062f2       _HeapDestroy@4             100072f2 f   kernel32:KERNEL32.dll
 0001:000062f8       _HeapAlloc@12              100072f8 f   kernel32:KERNEL32.dll
 0001:000062fe       _HeapFree@12               100072fe f   kernel32:KERNEL32.dll
 0001:00006304       _HeapValidate@12           10007304 f   kernel32:KERNEL32.dll
 0001:0000630a       _VirtualProtect@16         1000730a f   kernel32:KERNEL32.dll
 0001:00006310       _InitializeCriticalSection@4 10007310 f   kernel32:KERNEL32.dll
 0001:00006316       _DeleteCriticalSection@4   10007316 f   kernel32:KERNEL32.dll
 0001:0000631c       _GetSystemInfo@4           1000731c f   kernel32:KERNEL32.dll
 0001:00006322       _VirtualQueryEx@16         10007322 f   kernel32:KERNEL32.dll
 0001:00006328       _wsprintfA                 10007328 f   user32:USER32.dll
 0001:0000632e       _wvsprintfA@12             1000732e f   user32:USER32.dll
 0001:00006334       ?_Xbad_alloc@std@@YAXXZ    10007334 f   msvcprt:MSVCP110.dll
 0001:0000633a       ?_Xlength_error@std@@YAXPBD@Z 1000733a f   msvcprt:MSVCP110.dll
 0001:00006340       ?_Xout_of_range@std@@YAXPBD@Z 10007340 f   msvcprt:MSVCP110.dll
 0001:00006346       ?_Syserror_map@std@@YAPBDH@Z 10007346 f   msvcprt:MSVCP110.dll
 0001:0000634c       ?_Winerror_map@std@@YAPBDH@Z 1000734c f   msvcprt:MSVCP110.dll
 0001:00006352       ___CxxFrameHandler3        10007352 f   MSVCRT:MSVCR110.dll
 0001:00006360       __chkstk                   10007360 f   MSVCRT:chkstk.obj
 0001:00006360       __alloca_probe             10007360     MSVCRT:chkstk.obj
 0001:0000638c       _memset                    1000738c f   MSVCRT:MSVCR110.dll
 0001:00006392       ??3@YAXPAX@Z               10007392 f   MSVCRT:MSVCR110.dll
 0001:00006398       __purecall                 10007398 f   MSVCRT:MSVCR110.dll
 0001:0000639e       ??0type_info@@AAE@ABV0@@Z  1000739e f   MSVCRT:ti_inst.obj
 0001:000063a9       ??4type_info@@AAEAAV0@ABV0@@Z 100073a9 f   MSVCRT:ti_inst.obj
 0001:000063ae       ??_Etype_info@@UAEPAXI@Z   100073ae f i MSVCRT:ti_inst.obj
 0001:000063f8       ___isa_available_init      100073f8 f   MSVCRT:cpu_disp.obj
 0001:00006532       ??2@YAPAXI@Z               10007532 f   MSVCRT:MSVCR110.dll
 0001:00006538       ___atonexitinit            10007538 f   MSVCRT:atonexit.obj
 0001:00006574       __onexit                   10007574 f   MSVCRT:atonexit.obj
 0001:00006619       _atexit                    10007619 f   MSVCRT:atonexit.obj
 0001:0000662e       _memcpy                    1000762e f   MSVCRT:MSVCR110.dll
 0001:00006634       _strlen                    10007634 f   MSVCRT:MSVCR110.dll
 0001:0000663a       _memmove                   1000763a f   MSVCRT:MSVCR110.dll
 0001:00006640       __CxxThrowException@8      10007640 f   MSVCRT:MSVCR110.dll
 0001:00006646       ??_M@YGXPAXIHP6EX0@Z@Z     10007646 f   MSVCRT:ehvecdtr.obj
 0001:000066ce       ?__ArrayUnwind@@YGXPAXIHP6EX0@Z@Z 100076ce f   MSVCRT:ehvecdtr.obj
 0001:0000672c       ??1type_info@@UAE@XZ       1000772c f   MSVCRT:MSVCR110.dll
 0001:00006732       __lock                     10007732 f   MSVCRT:MSVCR110.dll
 0001:00006738       __unlock                   10007738 f   MSVCRT:MSVCR110.dll
 0001:0000673e       __calloc_crt               1000773e f   MSVCRT:MSVCR110.dll
 0001:00006744       ___dllonexit               10007744 f   MSVCRT:MSVCR110.dll
 0001:00006750       __SEH_prolog4              10007750 f   MSVCRT:sehprolg4.obj
 0001:00006795       __SEH_epilog4              10007795 f   MSVCRT:sehprolg4.obj
 0001:000067a9       __except_handler4          100077a9 f   MSVCRT:chandler4gs.obj
 0001:000067cc       ?terminate@@YAXXZ          100077cc f   MSVCRT:MSVCR110.dll
 0001:000067d2       @__security_check_cookie@4 100077d2 f   MSVCRT:secchk.obj
 0001:000067e2       __except_handler4_common   100077e2 f   MSVCRT:MSVCR110.dll
 0001:000067e8       ___raise_securityfailure   100077e8 f   MSVCRT:gs_report.obj
 0001:00006825       ___report_gsfailure        10007825 f   MSVCRT:gs_report.obj
 0001:0000691e       ___report_rangecheckfailure 1000791e f   MSVCRT:gs_report.obj
 0001:0000692a       ___report_securityfailure  1000792a f   MSVCRT:gs_report.obj
 0001:000069f8       ___report_securityfailureEx 100079f8 f   MSVCRT:gs_report.obj
 0001:00006b0c       __crt_debugger_hook        10007b0c f   MSVCRT:MSVCR110.dll
 0001:00006b12       ___crtUnhandledException   10007b12 f   MSVCRT:MSVCR110.dll
 0001:00006b18       ___crtTerminateProcess     10007b18 f   MSVCRT:MSVCR110.dll
 0001:00006b1e       _IsProcessorFeaturePresent@4 10007b1e f   kernel32:KERNEL32.dll
 0001:00006b24       _EncodePointer@4           10007b24 f   kernel32:KERNEL32.dll
 0001:00006b2a       _DecodePointer@4           10007b2a f   kernel32:KERNEL32.dll
 0001:00006b30       _IsDebuggerPresent@0       10007b30 f   kernel32:KERNEL32.dll
 0002:00000000       __imp__DeleteFileA@4       10008000     kernel32:KERNEL32.dll
 0002:00000004       __imp__GetFileAttributesA@4 10008004     kernel32:KERNEL32.dll
 0002:00000008       __imp__EnterCriticalSection@4 10008008     kernel32:KERNEL32.dll
 0002:0000000c       __imp__LeaveCriticalSection@4 1000800c     kernel32:KERNEL32.dll
 0002:00000010       __imp__lstrcmpiA@8         10008010     kernel32:KERNEL32.dll
 0002:00000014       __imp__lstrcpynA@12        10008014     kernel32:KERNEL32.dll
 0002:00000018       __imp__lstrcpyA@8          10008018     kernel32:KERNEL32.dll
 0002:0000001c       __imp__lstrlenA@4          1000801c     kernel32:KERNEL32.dll
 0002:00000020       __imp__OutputDebugStringA@4 10008020     kernel32:KERNEL32.dll
 0002:00000024       __imp__VirtualAlloc@16     10008024     kernel32:KERNEL32.dll
 0002:00000028       __imp__VirtualFree@12      10008028     kernel32:KERNEL32.dll
 0002:0000002c       __imp__DisableThreadLibraryCalls@4 1000802c     kernel32:KERNEL32.dll
 0002:00000030       __imp__GetModuleHandleA@4  10008030     kernel32:KERNEL32.dll
 0002:00000034       __imp__CreateFileA@28      10008034     kernel32:KERNEL32.dll
 0002:00000038       __imp__WriteFile@20        10008038     kernel32:KERNEL32.dll
 0002:0000003c       __imp__DebugBreak@0        1000803c     kernel32:KERNEL32.dll
 0002:00000040       __imp__CloseHandle@4       10008040     kernel32:KERNEL32.dll
 0002:00000044       __imp__GetProcessHeap@0    10008044     kernel32:KERNEL32.dll
 0002:00000048       __imp__GetProcessHeaps@8   10008048     kernel32:KERNEL32.dll
 0002:0000004c       __imp__HeapLock@4          1000804c     kernel32:KERNEL32.dll
 0002:00000050       __imp__HeapUnlock@4        10008050     kernel32:KERNEL32.dll
 0002:00000054       __imp__HeapWalk@8          10008054     kernel32:KERNEL32.dll
 0002:00000058       __imp__GetCurrentProcess@0 10008058     kernel32:KERNEL32.dll
 0002:0000005c       __imp__GetVersionExA@4     1000805c     kernel32:KERNEL32.dll
 0002:00000060       __imp__VirtualQuery@12     10008060     kernel32:KERNEL32.dll
 0002:00000064       __imp__GetProcAddress@8    10008064     kernel32:KERNEL32.dll
 0002:00000068       __imp__lstrcatA@8          10008068     kernel32:KERNEL32.dll
 0002:0000006c       __imp__LoadLibraryA@4      1000806c     kernel32:KERNEL32.dll
 0002:00000070       __imp__HeapCreate@12       10008070     kernel32:KERNEL32.dll
 0002:00000074       __imp__HeapDestroy@4       10008074     kernel32:KERNEL32.dll
 0002:00000078       __imp__HeapAlloc@12        10008078     kernel32:KERNEL32.dll
 0002:0000007c       __imp__HeapFree@12         1000807c     kernel32:KERNEL32.dll
 0002:00000080       __imp__HeapValidate@12     10008080     kernel32:KERNEL32.dll
 0002:00000084       __imp__VirtualProtect@16   10008084     kernel32:KERNEL32.dll
 0002:00000088       __imp__InitializeCriticalSection@4 10008088     kernel32:KERNEL32.dll
 0002:0000008c       __imp__DeleteCriticalSection@4 1000808c     kernel32:KERNEL32.dll
 0002:00000090       __imp__GetSystemInfo@4     10008090     kernel32:KERNEL32.dll
 0002:00000094       __imp__VirtualQueryEx@16   10008094     kernel32:KERNEL32.dll
 0002:00000098       __imp__DecodePointer@4     10008098     kernel32:KERNEL32.dll
 0002:0000009c       __imp__EncodePointer@4     1000809c     kernel32:KERNEL32.dll
 0002:000000a0       __imp__IsProcessorFeaturePresent@4 100080a0     kernel32:KERNEL32.dll
 0002:000000a4       __imp__IsDebuggerPresent@0 100080a4     kernel32:KERNEL32.dll
 0002:000000a8       \177KERNEL32_NULL_THUNK_DATA 100080a8     kernel32:KERNEL32.dll
 0002:000000ac       __imp_?_Xlength_error@std@@YAXPBD@Z 100080ac     msvcprt:MSVCP110.dll
 0002:000000b0       __imp_?_Xout_of_range@std@@YAXPBD@Z 100080b0     msvcprt:MSVCP110.dll
 0002:000000b4       __imp_?_Syserror_map@std@@YAPBDH@Z 100080b4     msvcprt:MSVCP110.dll
 0002:000000b8       __imp_?_Winerror_map@std@@YAPBDH@Z 100080b8     msvcprt:MSVCP110.dll
 0002:000000bc       __imp_?_Xbad_alloc@std@@YAXXZ 100080bc     msvcprt:MSVCP110.dll
 0002:000000c0       \177MSVCP110_NULL_THUNK_DATA 100080c0     msvcprt:MSVCP110.dll
 0002:000000c4       __imp__memset              100080c4     MSVCRT:MSVCR110.dll
 0002:000000c8       __imp_??3@YAXPAX@Z         100080c8     MSVCRT:MSVCR110.dll
 0002:000000cc       __imp___purecall           100080cc     MSVCRT:MSVCR110.dll
 0002:000000d0       __imp_??2@YAPAXI@Z         100080d0     MSVCRT:MSVCR110.dll
 0002:000000d4       __imp__memcpy              100080d4     MSVCRT:MSVCR110.dll
 0002:000000d8       __imp__strlen              100080d8     MSVCRT:MSVCR110.dll
 0002:000000dc       __imp__memmove             100080dc     MSVCRT:MSVCR110.dll
 0002:000000e0       __imp___CxxThrowException@8 100080e0     MSVCRT:MSVCR110.dll
 0002:000000e4       __imp____CxxFrameHandler3  100080e4     MSVCRT:MSVCR110.dll
 0002:000000e8       __imp___lock               100080e8     MSVCRT:MSVCR110.dll
 0002:000000ec       __imp___unlock             100080ec     MSVCRT:MSVCR110.dll
 0002:000000f0       __imp___calloc_crt         100080f0     MSVCRT:MSVCR110.dll
 0002:000000f4       __imp____dllonexit         100080f4     MSVCRT:MSVCR110.dll
 0002:000000f8       __imp___onexit             100080f8     MSVCRT:MSVCR110.dll
 0002:000000fc       __imp_?terminate@@YAXXZ    100080fc     MSVCRT:MSVCR110.dll
 0002:00000100       __imp___except_handler4_common 10008100     MSVCRT:MSVCR110.dll
 0002:00000104       __imp___crt_debugger_hook  10008104     MSVCRT:MSVCR110.dll
 0002:00000108       __imp____crtUnhandledException 10008108     MSVCRT:MSVCR110.dll
 0002:0000010c       __imp____crtTerminateProcess 1000810c     MSVCRT:MSVCR110.dll
 0002:00000110       __imp_??1type_info@@UAE@XZ 10008110     MSVCRT:MSVCR110.dll
 0002:00000114       \177MSVCR110_NULL_THUNK_DATA 10008114     MSVCRT:MSVCR110.dll
 0002:00000118       __imp__wsprintfA           10008118     user32:USER32.dll
 0002:0000011c       __imp__wvsprintfA@12       1000811c     user32:USER32.dll
 0002:00000120       \177USER32_NULL_THUNK_DATA 10008120     user32:USER32.dll
 0002:00000168       ??_C@_07MCAEODGB@Default?$AA@ 10008168     Memorylib.obj
 0002:00000170       ??_C@_07BJOIOONN@Strings?$AA@ 10008170     Memorylib.obj
 0002:00000178       ??_C@_00CNPNBAHC@?$AA@     10008178     Memorylib.obj
 0002:0000017c       ??_C@_0DG@JBJOOCCC@MemoryLib?3?5?$CIINFO?$CJ?5?3?5Small?5Pool?5?$CF@ 1000817c     MemorySmall.obj
 0002:000001b4       ??_C@_0BG@EHGOCKCA@vmdump?9workingset?4csv?$AA@ 100081b4     mmPeek.obj
 0002:000001cc       ??_C@_0BC@IDCHJEAP@vmdump?9blocks?4csv?$AA@ 100081cc     mmPeek.obj
 0002:000001e0       ??_C@_0BD@NMBHBMDH@vmdump?9regions?4csv?$AA@ 100081e0     mmPeek.obj
 0002:000001f4       ??_C@_0BB@JCGDPCLE@vmdump?9heaps?4csv?$AA@ 100081f4     mmPeek.obj
 0002:00000208       ??_C@_0BB@IGMAFNLO@vmdump?9pools?4csv?$AA@ 10008208     mmPeek.obj
 0002:0000021c       ??_C@_0BH@KNMEHFH@vmdump?9heapentries?4csv?$AA@ 1000821c     mmPeek.obj
 0002:00000234       ??_C@_0BH@HHBJHPFK@vmdump?9heapregions?4csv?$AA@ 10008234     mmPeek.obj
 0002:0000024c       ??_C@_0BH@CCAIIKP@vmdump?9smallchunks?4csv?$AA@ 1000824c     mmPeek.obj
 0002:00000264       ??_C@_02PCIJFNDE@?$AN?6?$AA@ 10008264     mmPeek.obj
 0002:00000268       ??_C@_01KICIPPFI@?2?$AA@   10008268     mmPeek.obj
 0002:0000026c       ??_C@_09LOPACEED@psapi?4dll?$AA@ 1000826c     mmPeek.obj
 0002:00000278       ??_C@_0BA@CJBKKPEL@EmptyWorkingSet?$AA@ 10008278     mmPeek.obj
 0002:00000288       ??_C@_0BD@CIEGPBCN@GetMappedFileNameA?$AA@ 10008288     mmPeek.obj
 0002:0000029c       ??_C@_0BF@OFAHHCBJ@GetModuleFileNameExA?$AA@ 1000829c     mmPeek.obj
 0002:000002b4       ??_C@_0BA@NCBDADEG@QueryWorkingSet?$AA@ 100082b4     mmPeek.obj
 0002:000002c4       ??_C@_04NEJBHOB@?$CF08x?$AA@ 100082c4     mmPeek.obj
 0002:000002cc       ??_C@_0BD@PINHKACJ@?$CF08x?0?5?$CF08x?0?5?$CFd?0?5?$CFd?$AA@ 100082cc     mmPeek.obj
 0002:000002e0       ??_C@_0BF@CNDFINHD@?$CF08x?0?5?$CFd?0?5?$CFd?0?5?$CFd?0?5?$CFs?$AA@ 100082e0     mmPeek.obj
 0002:000002f8       ??_C@_08LDLEFMMK@?$CF08x?0?5?$CFd?$AA@ 100082f8     mmPeek.obj
 0002:00000304       ??_C@_0BH@OCEJNDLB@?$CF08x?0?5?$CF08x?0?5?$CFd?0?5?$CFd?0?5?$CFd?$AA@ 10008304     mmPeek.obj
 0002:0000031c       ??_C@_07GAJLEDKM@0x?$CF08x?0?$AA@ 1000831c     mmPeek.obj
 0002:00000324       ??_C@_03DPLIHHLN@?$CFd?0?$AA@ 10008324     mmPeek.obj
 0002:00000328       ??_C@_05BFHEBJNP@?$CF02X?5?$AA@ 10008328     mmPeek.obj
 0002:00000330       ??_C@_01IHBHIGKO@?0?$AA@   10008330     mmPeek.obj
 0002:00000334       ??_C@_02HAOIJKIC@?$CFc?$AA@ 10008334     mmPeek.obj
 0002:00000338       ??_C@_08LGDHNIFM@?$CF08x?0?5?$CFs?$AA@ 10008338     mmPeek.obj
 0002:00000344       ??_C@_0BL@CDDCDOGI@?$CFx?0?5?$CFd?0?5?$CFd?0?5?$CFd?0?5?$CFd?0?5?$CFd?0?5?$CFs?$AA@ 10008344     mmPeek.obj
 0002:00000360       ??_C@_0BM@OPNJELD@address?0size?0bytes?0chars?0?$AN?6?$AA@ 10008360     mmPeek.obj
 0002:0000037c       ?MAGIC@MMPool@@2KB         1000837c     mmPool.obj
 0002:00000380       ?MAGIC@MMSnapshot@@0KB     10008380     mmPool.obj
 0002:00000384       ?MAGIC@MMSnapshotIterator@@0KB 10008384     mmPool.obj
 0002:000003a0       ??_7MMPoolBase@@6B@        100083a0     mmPool.obj
 0002:000003d4       ??_7MMPool@@6B@            100083d4     mmPool.obj
 0002:00000404       ??_C@_0DC@JEBKAKIJ@MemoryLib?3?5?$CIINFO?$CJ?5?3?5Pool?5?$CFs?0?5Lea@ 10008404     mmPool.obj
 0002:00000438       ??_C@_0DK@HIBBDNDK@MemoryLib?3?5?$CIINFO?$CJ?5?3?5Pool?5?$CFs?0?5max@ 10008438     mmPool.obj
 0002:00000480       __xmm@00000001000000010000000100000001 10008480     mmPool.obj
 0002:00000490       __xmm@00000003000000020000000100000000 10008490     mmPool.obj
 0002:000004a0       __xmm@00000014000000140000001400000014 100084a0     mmPool.obj
 0002:000004b0       ?MAGIC@MMPoolVM@@2KB       100084b0     mmPoolVM.obj
 0002:000004b8       ??_7MMPoolVM@@6B@          100084b8     mmPoolVM.obj
 0002:000004e8       ?radix@_Num_float_base@std@@2HB 100084e8     pch.obj
 0002:000004ec       ?is_signed@?$numeric_limits@D@std@@2_NB 100084ec     pch.obj
 0002:000004f0       ?digits@?$numeric_limits@D@std@@2HB 100084f0     pch.obj
 0002:000004f4       ?digits10@?$numeric_limits@D@std@@2HB 100084f4     pch.obj
 0002:000004f8       ?is_signed@?$numeric_limits@_W@std@@2_NB 100084f8     pch.obj
 0002:000004fc       ?digits@?$numeric_limits@_W@std@@2HB 100084fc     pch.obj
 0002:00000500       ?digits10@?$numeric_limits@_W@std@@2HB 10008500     pch.obj
 0002:00000504       ?is_modulo@?$numeric_limits@_N@std@@2_NB 10008504     pch.obj
 0002:00000505       ?is_signed@?$numeric_limits@_N@std@@2_NB 10008505     pch.obj
 0002:00000508       ?digits@?$numeric_limits@_N@std@@2HB 10008508     pch.obj
 0002:0000050c       ?digits10@?$numeric_limits@_N@std@@2HB 1000850c     pch.obj
 0002:00000510       ?is_signed@?$numeric_limits@C@std@@2_NB 10008510     pch.obj
 0002:00000514       ?digits@?$numeric_limits@C@std@@2HB 10008514     pch.obj
 0002:00000518       ?digits10@?$numeric_limits@C@std@@2HB 10008518     pch.obj
 0002:0000051c       ?is_signed@?$numeric_limits@E@std@@2_NB 1000851c     pch.obj
 0002:00000520       ?digits@?$numeric_limits@E@std@@2HB 10008520     pch.obj
 0002:00000524       ?digits10@?$numeric_limits@E@std@@2HB 10008524     pch.obj
 0002:00000528       ?is_signed@?$numeric_limits@F@std@@2_NB 10008528     pch.obj
 0002:0000052c       ?digits@?$numeric_limits@F@std@@2HB 1000852c     pch.obj
 0002:00000530       ?digits10@?$numeric_limits@F@std@@2HB 10008530     pch.obj
 0002:00000534       ?value@?$_Sizeof@U_Nil@std@@U12@U12@U12@U12@U12@U12@U12@@std@@2IB 10008534     pch.obj
 0002:00000538       ?is_signed@?$numeric_limits@G@std@@2_NB 10008538     pch.obj
 0002:0000053c       ?digits@?$numeric_limits@G@std@@2HB 1000853c     pch.obj
 0002:00000540       ?digits10@?$numeric_limits@G@std@@2HB 10008540     pch.obj
 0002:00000544       ?is_signed@?$numeric_limits@H@std@@2_NB 10008544     pch.obj
 0002:00000548       ?digits@?$numeric_limits@H@std@@2HB 10008548     pch.obj
 0002:0000054c       ?digits10@?$numeric_limits@H@std@@2HB 1000854c     pch.obj
 0002:00000550       ?is_signed@?$numeric_limits@I@std@@2_NB 10008550     pch.obj
 0002:00000554       ?digits@?$numeric_limits@I@std@@2HB 10008554     pch.obj
 0002:00000558       ?digits10@?$numeric_limits@I@std@@2HB 10008558     pch.obj
 0002:0000055c       ?value@?$integral_constant@_N$0A@@std@@2_NB 1000855c     pch.obj
 0002:0000055d       ?value@?$integral_constant@_N$00@std@@2_NB 1000855d     pch.obj
 0002:0000055e       ?is_signed@?$numeric_limits@J@std@@2_NB 1000855e     pch.obj
 0002:00000560       ?digits@?$numeric_limits@J@std@@2HB 10008560     pch.obj
 0002:00000564       ?digits10@?$numeric_limits@J@std@@2HB 10008564     pch.obj
 0002:00000568       ?is_signed@?$numeric_limits@K@std@@2_NB 10008568     pch.obj
 0002:0000056c       ?digits@?$numeric_limits@K@std@@2HB 1000856c     pch.obj
 0002:00000570       ?digits10@?$numeric_limits@K@std@@2HB 10008570     pch.obj
 0002:00000574       ?is_signed@?$numeric_limits@_J@std@@2_NB 10008574     pch.obj
 0002:00000578       ?digits@?$numeric_limits@_J@std@@2HB 10008578     pch.obj
 0002:0000057c       ?digits10@?$numeric_limits@_J@std@@2HB 1000857c     pch.obj
 0002:00000580       ?is_signed@?$numeric_limits@_K@std@@2_NB 10008580     pch.obj
 0002:00000584       ?digits@?$numeric_limits@_K@std@@2HB 10008584     pch.obj
 0002:00000588       ?digits10@?$numeric_limits@_K@std@@2HB 10008588     pch.obj
 0002:0000058c       ?digits@?$numeric_limits@M@std@@2HB 1000858c     pch.obj
 0002:00000590       ?digits10@?$numeric_limits@M@std@@2HB 10008590     pch.obj
 0002:00000594       ?max_digits10@?$numeric_limits@M@std@@2HB 10008594     pch.obj
 0002:00000598       ?value@?$_Sizeof@HU_Nil@std@@U12@U12@U12@U12@U12@U12@@std@@2IB 10008598     pch.obj
 0002:0000059c       ?max_exponent@?$numeric_limits@M@std@@2HB 1000859c     pch.obj
 0002:000005a0       ?max_exponent10@?$numeric_limits@M@std@@2HB 100085a0     pch.obj
 0002:000005a4       ?min_exponent@?$numeric_limits@M@std@@2HB 100085a4     pch.obj
 0002:000005a8       ?min_exponent10@?$numeric_limits@M@std@@2HB 100085a8     pch.obj
 0002:000005ac       ?digits@?$numeric_limits@N@std@@2HB 100085ac     pch.obj
 0002:000005b0       ?digits10@?$numeric_limits@N@std@@2HB 100085b0     pch.obj
 0002:000005b4       ?max_digits10@?$numeric_limits@N@std@@2HB 100085b4     pch.obj
 0002:000005b8       ?max_exponent@?$numeric_limits@N@std@@2HB 100085b8     pch.obj
 0002:000005bc       ?max_exponent10@?$numeric_limits@N@std@@2HB 100085bc     pch.obj
 0002:000005c0       ?min_exponent@?$numeric_limits@N@std@@2HB 100085c0     pch.obj
 0002:000005c4       ?min_exponent10@?$numeric_limits@N@std@@2HB 100085c4     pch.obj
 0002:000005c8       ?digits@?$numeric_limits@O@std@@2HB 100085c8     pch.obj
 0002:000005cc       ?digits10@?$numeric_limits@O@std@@2HB 100085cc     pch.obj
 0002:000005d0       ?max_digits10@?$numeric_limits@O@std@@2HB 100085d0     pch.obj
 0002:000005d4       ?max_exponent@?$numeric_limits@O@std@@2HB 100085d4     pch.obj
 0002:000005d8       ?max_exponent10@?$numeric_limits@O@std@@2HB 100085d8     pch.obj
 0002:000005dc       ?min_exponent@?$numeric_limits@O@std@@2HB 100085dc     pch.obj
 0002:000005e0       ?min_exponent10@?$numeric_limits@O@std@@2HB 100085e0     pch.obj
 0002:000005e4       ?value@?$integral_constant@I$0A@@std@@2IB 100085e4     pch.obj
 0002:000005e8       ?has_denorm@_Num_base@std@@2W4float_denorm_style@2@B 100085e8     pch.obj
 0002:000005ec       ?has_denorm_loss@_Num_base@std@@2_NB 100085ec     pch.obj
 0002:000005ed       ?has_infinity@_Num_base@std@@2_NB 100085ed     pch.obj
 0002:000005ee       ?has_quiet_NaN@_Num_base@std@@2_NB 100085ee     pch.obj
 0002:000005ef       ?has_signaling_NaN@_Num_base@std@@2_NB 100085ef     pch.obj
 0002:000005f0       ?is_bounded@_Num_base@std@@2_NB 100085f0     pch.obj
 0002:000005f1       ?is_exact@_Num_base@std@@2_NB 100085f1     pch.obj
 0002:000005f2       ?is_iec559@_Num_base@std@@2_NB 100085f2     pch.obj
 0002:000005f3       ?is_integer@_Num_base@std@@2_NB 100085f3     pch.obj
 0002:000005f4       ?is_modulo@_Num_base@std@@2_NB 100085f4     pch.obj
 0002:000005f5       ?is_signed@_Num_base@std@@2_NB 100085f5     pch.obj
 0002:000005f6       ?is_specialized@_Num_base@std@@2_NB 100085f6     pch.obj
 0002:000005f7       ?tinyness_before@_Num_base@std@@2_NB 100085f7     pch.obj
 0002:000005f8       ?traps@_Num_base@std@@2_NB 100085f8     pch.obj
 0002:000005fc       ?round_style@_Num_base@std@@2W4float_round_style@2@B 100085fc     pch.obj
 0002:00000600       ?digits@_Num_base@std@@2HB 10008600     pch.obj
 0002:00000604       ?digits10@_Num_base@std@@2HB 10008604     pch.obj
 0002:00000608       ?max_digits10@_Num_base@std@@2HB 10008608     pch.obj
 0002:0000060c       ?max_exponent@_Num_base@std@@2HB 1000860c     pch.obj
 0002:00000610       ?max_exponent10@_Num_base@std@@2HB 10008610     pch.obj
 0002:00000614       ?min_exponent@_Num_base@std@@2HB 10008614     pch.obj
 0002:00000618       ?min_exponent10@_Num_base@std@@2HB 10008618     pch.obj
 0002:0000061c       ?radix@_Num_base@std@@2HB  1000861c     pch.obj
 0002:00000620       ?is_bounded@_Num_int_base@std@@2_NB 10008620     pch.obj
 0002:00000621       ?is_exact@_Num_int_base@std@@2_NB 10008621     pch.obj
 0002:00000622       ?is_integer@_Num_int_base@std@@2_NB 10008622     pch.obj
 0002:00000623       ?is_modulo@_Num_int_base@std@@2_NB 10008623     pch.obj
 0002:00000624       ?is_specialized@_Num_int_base@std@@2_NB 10008624     pch.obj
 0002:00000628       ?radix@_Num_int_base@std@@2HB 10008628     pch.obj
 0002:0000062c       ?has_denorm@_Num_float_base@std@@2W4float_denorm_style@2@B 1000862c     pch.obj
 0002:00000630       ?has_denorm_loss@_Num_float_base@std@@2_NB 10008630     pch.obj
 0002:00000631       ?has_infinity@_Num_float_base@std@@2_NB 10008631     pch.obj
 0002:00000632       ?has_quiet_NaN@_Num_float_base@std@@2_NB 10008632     pch.obj
 0002:00000633       ?has_signaling_NaN@_Num_float_base@std@@2_NB 10008633     pch.obj
 0002:00000634       ?is_bounded@_Num_float_base@std@@2_NB 10008634     pch.obj
 0002:00000635       ?is_exact@_Num_float_base@std@@2_NB 10008635     pch.obj
 0002:00000636       ?is_iec559@_Num_float_base@std@@2_NB 10008636     pch.obj
 0002:00000637       ?is_integer@_Num_float_base@std@@2_NB 10008637     pch.obj
 0002:00000638       ?is_modulo@_Num_float_base@std@@2_NB 10008638     pch.obj
 0002:00000639       ?is_signed@_Num_float_base@std@@2_NB 10008639     pch.obj
 0002:0000063a       ?is_specialized@_Num_float_base@std@@2_NB 1000863a     pch.obj
 0002:0000063b       ?tinyness_before@_Num_float_base@std@@2_NB 1000863b     pch.obj
 0002:0000063c       ?traps@_Num_float_base@std@@2_NB 1000863c     pch.obj
 0002:00000640       ?round_style@_Num_float_base@std@@2W4float_round_style@2@B 10008640     pch.obj
 0002:00000644       ?collate@?$_Locbase@H@std@@2HB 10008644     mmgr.obj
 0002:00000648       ?ctype@?$_Locbase@H@std@@2HB 10008648     mmgr.obj
 0002:0000064c       ?monetary@?$_Locbase@H@std@@2HB 1000864c     mmgr.obj
 0002:00000650       ?numeric@?$_Locbase@H@std@@2HB 10008650     mmgr.obj
 0002:00000654       ?time@?$_Locbase@H@std@@2HB 10008654     mmgr.obj
 0002:00000658       ?messages@?$_Locbase@H@std@@2HB 10008658     mmgr.obj
 0002:0000065c       ?all@?$_Locbase@H@std@@2HB 1000865c     mmgr.obj
 0002:00000660       ?none@?$_Locbase@H@std@@2HB 10008660     mmgr.obj
 0002:00000664       ?skipws@?$_Iosb@H@std@@2W4_Fmtflags@12@B 10008664     mmgr.obj
 0002:00000668       ?unitbuf@?$_Iosb@H@std@@2W4_Fmtflags@12@B 10008668     mmgr.obj
 0002:0000066c       ?uppercase@?$_Iosb@H@std@@2W4_Fmtflags@12@B 1000866c     mmgr.obj
 0002:00000670       ?showbase@?$_Iosb@H@std@@2W4_Fmtflags@12@B 10008670     mmgr.obj
 0002:00000674       ?showpoint@?$_Iosb@H@std@@2W4_Fmtflags@12@B 10008674     mmgr.obj
 0002:00000678       ?showpos@?$_Iosb@H@std@@2W4_Fmtflags@12@B 10008678     mmgr.obj
 0002:0000067c       ?left@?$_Iosb@H@std@@2W4_Fmtflags@12@B 1000867c     mmgr.obj
 0002:00000680       ?right@?$_Iosb@H@std@@2W4_Fmtflags@12@B 10008680     mmgr.obj
 0002:00000684       ?internal@?$_Iosb@H@std@@2W4_Fmtflags@12@B 10008684     mmgr.obj
 0002:00000688       ?dec@?$_Iosb@H@std@@2W4_Fmtflags@12@B 10008688     mmgr.obj
 0002:0000068c       ?oct@?$_Iosb@H@std@@2W4_Fmtflags@12@B 1000868c     mmgr.obj
 0002:00000690       ?hex@?$_Iosb@H@std@@2W4_Fmtflags@12@B 10008690     mmgr.obj
 0002:00000694       ?scientific@?$_Iosb@H@std@@2W4_Fmtflags@12@B 10008694     mmgr.obj
 0002:00000698       ?fixed@?$_Iosb@H@std@@2W4_Fmtflags@12@B 10008698     mmgr.obj
 0002:0000069c       ?hexfloat@?$_Iosb@H@std@@2W4_Fmtflags@12@B 1000869c     mmgr.obj
 0002:000006a0       ?boolalpha@?$_Iosb@H@std@@2W4_Fmtflags@12@B 100086a0     mmgr.obj
 0002:000006a4       ?_Stdio@?$_Iosb@H@std@@2W4_Fmtflags@12@B 100086a4     mmgr.obj
 0002:000006a8       ?adjustfield@?$_Iosb@H@std@@2W4_Fmtflags@12@B 100086a8     mmgr.obj
 0002:000006ac       ?basefield@?$_Iosb@H@std@@2W4_Fmtflags@12@B 100086ac     mmgr.obj
 0002:000006b0       ?floatfield@?$_Iosb@H@std@@2W4_Fmtflags@12@B 100086b0     mmgr.obj
 0002:000006b4       ?goodbit@?$_Iosb@H@std@@2W4_Iostate@12@B 100086b4     mmgr.obj
 0002:000006b8       ?eofbit@?$_Iosb@H@std@@2W4_Iostate@12@B 100086b8     mmgr.obj
 0002:000006bc       ?failbit@?$_Iosb@H@std@@2W4_Iostate@12@B 100086bc     mmgr.obj
 0002:000006c0       ?badbit@?$_Iosb@H@std@@2W4_Iostate@12@B 100086c0     mmgr.obj
 0002:000006c4       ?_Hardfail@?$_Iosb@H@std@@2W4_Iostate@12@B 100086c4     mmgr.obj
 0002:000006c8       ?in@?$_Iosb@H@std@@2W4_Openmode@12@B 100086c8     mmgr.obj
 0002:000006cc       ?out@?$_Iosb@H@std@@2W4_Openmode@12@B 100086cc     mmgr.obj
 0002:000006d0       ?ate@?$_Iosb@H@std@@2W4_Openmode@12@B 100086d0     mmgr.obj
 0002:000006d4       ?app@?$_Iosb@H@std@@2W4_Openmode@12@B 100086d4     mmgr.obj
 0002:000006d8       ?trunc@?$_Iosb@H@std@@2W4_Openmode@12@B 100086d8     mmgr.obj
 0002:000006dc       ?_Nocreate@?$_Iosb@H@std@@2W4_Openmode@12@B 100086dc     mmgr.obj
 0002:000006e0       ?_Noreplace@?$_Iosb@H@std@@2W4_Openmode@12@B 100086e0     mmgr.obj
 0002:000006e4       ?binary@?$_Iosb@H@std@@2W4_Openmode@12@B 100086e4     mmgr.obj
 0002:000006e8       ?beg@?$_Iosb@H@std@@2W4_Seekdir@12@B 100086e8     mmgr.obj
 0002:000006ec       ?cur@?$_Iosb@H@std@@2W4_Seekdir@12@B 100086ec     mmgr.obj
 0002:000006f0       ?end@?$_Iosb@H@std@@2W4_Seekdir@12@B 100086f0     mmgr.obj
 0002:000006f4       ?_Stream_err@failure@ios_base@std@@0W4io_errc@43@B 100086f4     mmgr.obj
 0002:000006fc       ??_7error_category@std@@6B@ 100086fc     mmgr.obj
 0002:00000718       ??_7_Generic_error_category@std@@6B@ 10008718     mmgr.obj
 0002:00000730       ??_C@_07DCLBNMLN@generic?$AA@ 10008730     mmgr.obj
 0002:00000738       ??_C@_0O@BFJCFAAK@unknown?5error?$AA@ 10008738     mmgr.obj
 0002:0000074c       ??_7_Iostream_error_category@std@@6B@ 1000874c     mmgr.obj
 0002:00000764       ??_C@_08LLGCOLLL@iostream?$AA@ 10008764     mmgr.obj
 0002:00000770       ??_C@_0BG@PADBLCHM@iostream?5stream?5error?$AA@ 10008770     mmgr.obj
 0002:0000078c       ??_7_System_error_category@std@@6B@ 1000878c     mmgr.obj
 0002:000007a4       ??_C@_06FHFOAHML@system?$AA@ 100087a4     mmgr.obj
 0002:000007ac       ??_C@_0BI@CFPLBAOH@invalid?5string?5position?$AA@ 100087ac     mmgr.obj
 0002:000007c4       ??_C@_0BA@JFNIOLAK@string?5too?5long?$AA@ 100087c4     mmgr.obj
 0002:000007d8       ??_7type_info@@6B@         100087d8     MSVCRT:ti_inst.obj
 0002:000007e8       __load_config_used         100087e8     MSVCRT:loadcfg.obj
 0002:0000089c       ??_R4MMPoolBase@@6B@       1000889c     mmPool.obj
 0002:000008b0       ??_R3MMPoolBase@@8         100088b0     mmPool.obj
 0002:000008c0       ??_R2MMPoolBase@@8         100088c0     mmPool.obj
 0002:000008c8       ??_R1A@?0A@EA@MMPoolBase@@8 100088c8     mmPool.obj
 0002:000008e4       ??_R4MMPool@@6B@           100088e4     mmPool.obj
 0002:000008f8       ??_R3MMPool@@8             100088f8     mmPool.obj
 0002:00000908       ??_R2MMPool@@8             10008908     mmPool.obj
 0002:00000914       ??_R1A@?0A@EA@MMPool@@8    10008914     mmPool.obj
 0002:00000930       ??_R4MMPoolVM@@6B@         10008930     mmPoolVM.obj
 0002:00000944       ??_R3MMPoolVM@@8           10008944     mmPoolVM.obj
 0002:00000954       ??_R2MMPoolVM@@8           10008954     mmPoolVM.obj
 0002:00000960       ??_R1A@?0A@EA@MMPoolVM@@8  10008960     mmPoolVM.obj
 0002:0000097c       ??_R4error_category@std@@6B@ 1000897c     mmgr.obj
 0002:00000990       ??_R3error_category@std@@8 10008990     mmgr.obj
 0002:000009a0       ??_R2error_category@std@@8 100089a0     mmgr.obj
 0002:000009a8       ??_R1A@?0A@EA@error_category@std@@8 100089a8     mmgr.obj
 0002:000009c4       ??_R4_Generic_error_category@std@@6B@ 100089c4     mmgr.obj
 0002:000009d8       ??_R3_Generic_error_category@std@@8 100089d8     mmgr.obj
 0002:000009e8       ??_R2_Generic_error_category@std@@8 100089e8     mmgr.obj
 0002:000009f4       ??_R1A@?0A@EA@_Generic_error_category@std@@8 100089f4     mmgr.obj
 0002:00000a10       ??_R4_Iostream_error_category@std@@6B@ 10008a10     mmgr.obj
 0002:00000a24       ??_R3_Iostream_error_category@std@@8 10008a24     mmgr.obj
 0002:00000a34       ??_R2_Iostream_error_category@std@@8 10008a34     mmgr.obj
 0002:00000a44       ??_R1A@?0A@EA@_Iostream_error_category@std@@8 10008a44     mmgr.obj
 0002:00000a60       ??_R4_System_error_category@std@@6B@ 10008a60     mmgr.obj
 0002:00000a74       ??_R3_System_error_category@std@@8 10008a74     mmgr.obj
 0002:00000a84       ??_R2_System_error_category@std@@8 10008a84     mmgr.obj
 0002:00000a94       ??_R1A@?0A@EA@_System_error_category@std@@8 10008a94     mmgr.obj
 0002:00000ab0       ??_R4type_info@@6B@        10008ab0     MSVCRT:ti_inst.obj
 0002:00000ac4       ??_R3type_info@@8          10008ac4     MSVCRT:ti_inst.obj
 0002:00000ad4       ??_R2type_info@@8          10008ad4     MSVCRT:ti_inst.obj
 0002:00000adc       ??_R1A@?0A@EA@type_info@@8 10008adc     MSVCRT:ti_inst.obj
 0002:00000b00       ___safe_se_handler_table   10008b00     <linker-defined>
 0002:00001204       __IMPORT_DESCRIPTOR_KERNEL32 10009204     kernel32:KERNEL32.dll
 0002:00001218       __IMPORT_DESCRIPTOR_USER32 10009218     user32:USER32.dll
 0002:0000122c       __IMPORT_DESCRIPTOR_MSVCP110 1000922c     msvcprt:MSVCP110.dll
 0002:00001240       __IMPORT_DESCRIPTOR_MSVCR110 10009240     MSVCRT:MSVCR110.dll
 0002:00001254       __NULL_IMPORT_DESCRIPTOR   10009254     kernel32:KERNEL32.dll
 0003:00000000       ?REPORT@MPeekRegion@@2PBDB 1000b000     mmPeek.obj
 0003:00000004       ?REPORT@MPeekBlock@@2PBDB  1000b004     mmPeek.obj
 0003:00000008       ?REPORT@MPeekWSPage@@2PBDB 1000b008     mmPeek.obj
 0003:0000000c       ?REPORT@MPeekHeap@@2PBDB   1000b00c     mmPeek.obj
 0003:00000010       ?REPORT@MPeekPool@@2PBDB   1000b010     mmPeek.obj
 0003:00000014       ?REPORT@MPeekHeapEntry@@2PBDB 1000b014     mmPeek.obj
 0003:00000018       ?REPORT@MPeekHeapRegion@@2PBDB 1000b018     mmPeek.obj
 0003:0000001c       ?REPORT@MPeekSmallChunk@@2PBDB 1000b01c     mmPeek.obj
 0003:00000024       ??_R0?AVMMPoolBase@@@8     1000b024     mmPool.obj
 0003:00000040       ??_R0?AVMMPool@@@8         1000b040     mmPool.obj
 0003:00000058       ??_R0?AVMMPoolVM@@@8       1000b058     mmPoolVM.obj
 0003:00000070       ?_Generic_object@?$_Error_objects@H@std@@2V_Generic_error_category@2@A 1000b070     mmgr.obj
 0003:00000074       ?_Iostream_object@?$_Error_objects@H@std@@2V_Iostream_error_category@2@A 1000b074     mmgr.obj
 0003:00000078       ?_System_object@?$_Error_objects@H@std@@2V_System_error_category@2@A 1000b078     mmgr.obj
 0003:0000007c       ??_R0?AVerror_category@std@@@8 1000b07c     mmgr.obj
 0003:000000a0       ??_R0?AV_Generic_error_category@std@@@8 1000b0a0     mmgr.obj
 0003:000000cc       ??_R0?AV_Iostream_error_category@std@@@8 1000b0cc     mmgr.obj
 0003:000000f8       ??_R0?AV_System_error_category@std@@@8 1000b0f8     mmgr.obj
 0003:00000130       ??_R0?AVtype_info@@@8      1000b130     MSVCRT:ti_inst.obj
 0003:00000148       ___isa_enabled             1000b148     MSVCRT:cpu_disp.obj
 0003:00000150       ___security_cookie         1000b150     MSVCRT:gs_cookie.obj
 0003:00000154       ___security_cookie_complement 1000b154     MSVCRT:gs_cookie.obj
 0003:00000164       ?s_usercbAlloc@@3P6GXABQAU_HMEMPOOL@@ABUMEMBLOCKINFO@@@ZA 1000b164     Memorylib.obj
 0003:0000026c       ?s_llhead@SmallInternals@?A0x79a48f2f@@0PAV12@A 1000b26c     MemorySmall.obj
 0003:00000270       ?useless@@3HA              1000b270     mmCRT.obj
 0003:00000288       ?maxqty@MMAllocInfo@@2IA   1000b288     mmPool.obj
 0003:0000028c       ?maxskip@MMAllocInfo@@2IA  1000b28c     mmPool.obj
 0003:00000290       ?maxskip@MMAllocTrace@@2IA 1000b290     mmPool.obj
 0003:000002a0       ___isa_available_default   1000b2a0     mmPool.obj
 0003:000002a4       ?s_instance@Internals@MMPoolVM@@0PAV12@A 1000b2a4     mmPoolVM.obj
 0003:000002a8       ?s_REGIONHEAP@?A0xbfaf6e17@@3PAXA 1000b2a8     mmPoolVM.obj
 0003:000002ac       ?g_GlobalLock@@3PAVMMThreadLockObj@@A 1000b2ac     mmThreadLock.obj
 0003:000022c8       ___@@_PchSym_@00@UsrxplibRkxhsrkUslnvdliowCxozhhrxUhixUrmgvinvwrzgvUhszivwUnvnlibUivovzhvUlyqUkxsOlyq@BE38CBA9A89F5D7C 1000d2c8     pch.obj
 0003:000022d8       ___isa_available           1000d2d8     MSVCRT:cpu_disp.obj
 0003:000022dc       ___favor                   1000d2dc     MSVCRT:cpu_disp.obj
 0003:00002600       ___onexitend               1000d600     <common>
 0003:00002604       ___onexitbegin             1000d604     <common>

 entry point at        0000:00000000

 Static symbols

 0000:fffef000       .debug$S                   10000000     MSVCRT:MSVCR110.dll
 0000:fffef000       .debug$S                   10000000     MSVCRT:MSVCR110.dll
 0000:fffef000       .debug$S                   10000000     MSVCRT:MSVCR110.dll
 0000:fffef000       .debug$S                   10000000     MSVCRT:MSVCR110.dll
 0000:fffef000       .debug$S                   10000000     MSVCRT:MSVCR110.dll
 0000:fffef000       .debug$S                   10000000     MSVCRT:MSVCR110.dll
 0000:fffef000       .debug$S                   10000000     MSVCRT:MSVCR110.dll
 0000:fffef000       .debug$S                   10000000     MSVCRT:MSVCR110.dll
 0000:fffef000       .debug$S                   10000000     MSVCRT:MSVCR110.dll
 0000:fffef000       .debug$S                   10000000     MSVCRT:MSVCR110.dll
 0000:fffef000       .debug$S                   10000000     MSVCRT:MSVCR110.dll
 0000:fffef000       .debug$S                   10000000     MSVCRT:MSVCR110.dll
 0000:fffef000       .debug$S                   10000000     MSVCRT:MSVCR110.dll
 0000:fffef000       .debug$S                   10000000     MSVCRT:MSVCR110.dll
 0000:fffef000       .debug$S                   10000000     MSVCRT:MSVCR110.dll
 0000:fffef000       .debug$S                   10000000     MSVCRT:MSVCR110.dll
 0000:fffef000       .debug$S                   10000000     MSVCRT:MSVCR110.dll
 0000:fffef000       .debug$S                   10000000     MSVCRT:MSVCR110.dll
 0000:fffef000       .debug$S                   10000000     MSVCRT:MSVCR110.dll
 0000:fffef000       .debug$S                   10000000     MSVCRT:MSVCR110.dll
 0000:fffef000       .debug$S                   10000000     kernel32:KERNEL32.dll
 0000:fffef000       .debug$S                   10000000     kernel32:KERNEL32.dll
 0000:fffef000       .debug$S                   10000000     kernel32:KERNEL32.dll
 0000:fffef000       .debug$S                   10000000     msvcprt:MSVCP110.dll
 0000:fffef000       .debug$S                   10000000     msvcprt:MSVCP110.dll
 0000:fffef000       .debug$S                   10000000     msvcprt:MSVCP110.dll
 0000:fffef000       .debug$S                   10000000     msvcprt:MSVCP110.dll
 0000:fffef000       .debug$S                   10000000     msvcprt:MSVCP110.dll
 0000:fffef000       .debug$S                   10000000     user32:USER32.dll
 0000:fffef000       .debug$S                   10000000     user32:USER32.dll
 0000:fffef000       .debug$S                   10000000     kernel32:KERNEL32.dll
 0000:fffef000       .debug$S                   10000000     kernel32:KERNEL32.dll
 0000:fffef000       .debug$S                   10000000     kernel32:KERNEL32.dll
 0000:fffef000       .debug$S                   10000000     kernel32:KERNEL32.dll
 0000:fffef000       .debug$S                   10000000     kernel32:KERNEL32.dll
 0000:fffef000       .debug$S                   10000000     kernel32:KERNEL32.dll
 0000:fffef000       .debug$S                   10000000     kernel32:KERNEL32.dll
 0000:fffef000       .debug$S                   10000000     kernel32:KERNEL32.dll
 0000:fffef000       .debug$S                   10000000     kernel32:KERNEL32.dll
 0000:fffef000       .debug$S                   10000000     kernel32:KERNEL32.dll
 0000:fffef000       .debug$S                   10000000     kernel32:KERNEL32.dll
 0000:fffef000       .debug$S                   10000000     kernel32:KERNEL32.dll
 0000:fffef000       .debug$S                   10000000     kernel32:KERNEL32.dll
 0000:fffef000       .debug$S                   10000000     kernel32:KERNEL32.dll
 0000:fffef000       .debug$S                   10000000     kernel32:KERNEL32.dll
 0000:fffef000       .debug$S                   10000000     kernel32:KERNEL32.dll
 0000:fffef000       .debug$S                   10000000     kernel32:KERNEL32.dll
 0000:fffef000       .debug$S                   10000000     kernel32:KERNEL32.dll
 0000:fffef000       .debug$S                   10000000     kernel32:KERNEL32.dll
 0000:fffef000       .debug$S                   10000000     kernel32:KERNEL32.dll
 0000:fffef000       .debug$S                   10000000     kernel32:KERNEL32.dll
 0000:fffef000       .debug$S                   10000000     kernel32:KERNEL32.dll
 0000:fffef000       .debug$S                   10000000     kernel32:KERNEL32.dll
 0000:fffef000       .debug$S                   10000000     kernel32:KERNEL32.dll
 0000:fffef000       .debug$S                   10000000     kernel32:KERNEL32.dll
 0000:fffef000       .debug$S                   10000000     kernel32:KERNEL32.dll
 0000:fffef000       .debug$S                   10000000     kernel32:KERNEL32.dll
 0000:fffef000       .debug$S                   10000000     kernel32:KERNEL32.dll
 0000:fffef000       .debug$S                   10000000     kernel32:KERNEL32.dll
 0000:fffef000       .debug$S                   10000000     kernel32:KERNEL32.dll
 0000:fffef000       .debug$S                   10000000     kernel32:KERNEL32.dll
 0000:fffef000       .debug$S                   10000000     kernel32:KERNEL32.dll
 0000:fffef000       .debug$S                   10000000     kernel32:KERNEL32.dll
 0000:fffef000       .debug$S                   10000000     kernel32:KERNEL32.dll
 0000:fffef000       .debug$S                   10000000     kernel32:KERNEL32.dll
 0000:fffef000       .debug$S                   10000000     kernel32:KERNEL32.dll
 0000:fffef000       .debug$S                   10000000     kernel32:KERNEL32.dll
 0000:fffef000       .debug$S                   10000000     kernel32:KERNEL32.dll
 0000:fffef000       .debug$S                   10000000     kernel32:KERNEL32.dll
 0001:00000040       ?ConvertMemoryPool@@YGPAVMMPoolBase@@PAX@Z 10001040 f   Memorylib.obj
 0001:00000060       ?CreateMemoryPool@@YGPAVMMPoolBase@@PBDI@Z 10001060 f   Memorylib.obj
 0001:000022c0       ?BuildFName@@YGXPADPBD1@Z  100032c0 f   mmPeek.obj
 0001:00002310       ?DumpHeapEntryToFile@@YGXPAXPBXI@Z 10003310 f   mmPeek.obj
 0001:00002450       ?DumpHeapToFile@@YGXPAX0@Z 10003450 f   mmPeek.obj
 0001:00002600       ?DumpHeaps@@YG_NPAXPBD11@Z 10003600 f   mmPeek.obj
 0001:00002860       ?DumpMemBlocks@@YG_NPAXAAVMPeekFile@?A0x85ca0ab9@@PBXK@Z 10003860 f   mmPeek.obj
 0001:0000296c       $LN30                      1000396c     mmPeek.obj
 0001:0000298c       $LN24                      1000398c     mmPeek.obj
 0001:00002a10       ?DumpMemRegions@@YG_NPAXPBD1@Z 10003a10 f   mmPeek.obj
 0001:00002c20       ?DumpWorkingSet@@YG_NPAXPBD@Z 10003c20 f   mmPeek.obj
 0001:00002d60       ?IsCharPrint@@YG_ND@Z      10003d60 f   mmPeek.obj
 0001:00002da4       $LN12                      10003da4     mmPeek.obj
 0001:00002dac       $LN10                      10003dac     mmPeek.obj
 0001:00002df0       ?MPeekInitialize@@YG_NXZ   10003df0 f   mmPeek.obj
 0001:00003480       ?ShrinkWS@@YG_NPAX_N@Z     10004480 f   mmPeek.obj
 0001:00004540       ?hashBlock@@YGKPBXI@Z      10005540 f   mmPool.obj
 0001:00005400       ?VMQueryHelp@@YGHPAXPBXPAUVMQUERY_HELP@@@Z 10006400 f   VMQuery.obj
 0001:0000589c       __catch$?_Copy@?$basic_string@DU?$char_traits@D@std@@V?$allocator@D@2@@std@@QAEXII@Z$0 1000689c f i mmgr.obj
 0001:000058d9       __catch$?_Copy@?$basic_string@DU?$char_traits@D@std@@V?$allocator@D@2@@std@@QAEXII@Z$1 100068d9 f i mmgr.obj
 0001:00006360       $$000000                   10007360     MSVCRT:chkstk.obj
 0001:000066b5       ?ArrayUnwindFilter@@YAHPAU_EXCEPTION_POINTERS@@@Z 100076b5 f   MSVCRT:ehvecdtr.obj
 0001:00006750       $$000000                   10007750     MSVCRT:sehprolg4.obj
 0001:00006b40       __unwindfunclet$?MemCRTAlloc@@YGPAXIH@Z$0 10007b40 f   Memorylib.obj
 0001:00006b48       __ehhandler$?MemCRTAlloc@@YGPAXIH@Z 10007b48 f   Memorylib.obj
 0001:00006b60       __unwindfunclet$?MemCRTFree@@YGXPAXH@Z$0 10007b60 f   Memorylib.obj
 0001:00006b68       __ehhandler$?MemCRTFree@@YGXPAXH@Z 10007b68 f   Memorylib.obj
 0001:00006b80       __unwindfunclet$?MemPoolAlloc@@YGPAXPAU_HMEMPOOL@@I@Z$0 10007b80 f   Memorylib.obj
 0001:00006b88       __ehhandler$?MemPoolAlloc@@YGPAXPAU_HMEMPOOL@@I@Z 10007b88 f   Memorylib.obj
 0001:00006ba0       __unwindfunclet$?MemPoolCreate@@YGPAU_HMEMPOOL@@PBDI@Z$0 10007ba0 f   Memorylib.obj
 0001:00006ba8       __ehhandler$?MemPoolCreate@@YGPAU_HMEMPOOL@@PBDI@Z 10007ba8 f   Memorylib.obj
 0001:00006bc0       __unwindfunclet$?MemPoolDestroy@@YGXPAU_HMEMPOOL@@@Z$0 10007bc0 f   Memorylib.obj
 0001:00006bc8       __ehhandler$?MemPoolDestroy@@YGXPAU_HMEMPOOL@@@Z 10007bc8 f   Memorylib.obj
 0001:00006be0       __unwindfunclet$?MemPoolFree@@YGXPAU_HMEMPOOL@@PAX@Z$0 10007be0 f   Memorylib.obj
 0001:00006be8       __ehhandler$?MemPoolFree@@YGXPAU_HMEMPOOL@@PAX@Z 10007be8 f   Memorylib.obj
 0001:00006c00       __unwindfunclet$?MemPoolLock@@YGXPAU_HMEMPOOL@@@Z$0 10007c00 f   Memorylib.obj
 0001:00006c08       __ehhandler$?MemPoolLock@@YGXPAU_HMEMPOOL@@@Z 10007c08 f   Memorylib.obj
 0001:00006c20       __unwindfunclet$?MemPoolName@@YGPBDPAU_HMEMPOOL@@@Z$0 10007c20 f   Memorylib.obj
 0001:00006c28       __ehhandler$?MemPoolName@@YGPBDPAU_HMEMPOOL@@@Z 10007c28 f   Memorylib.obj
 0001:00006c40       __unwindfunclet$?MemPoolSize@@YGXPAU_HMEMPOOL@@AAI1@Z$0 10007c40 f   Memorylib.obj
 0001:00006c48       __ehhandler$?MemPoolSize@@YGXPAU_HMEMPOOL@@AAI1@Z 10007c48 f   Memorylib.obj
 0001:00006c60       __unwindfunclet$?MemPoolSnapshot@@YGPAU_HMEMPOOLSHOT@@PAU_HMEMPOOL@@@Z$0 10007c60 f   Memorylib.obj
 0001:00006c68       __ehhandler$?MemPoolSnapshot@@YGPAU_HMEMPOOLSHOT@@PAU_HMEMPOOL@@@Z 10007c68 f   Memorylib.obj
 0001:00006c80       __unwindfunclet$?MemPoolSnapshotDestroy@@YGXPAU_HMEMPOOLSHOT@@@Z$0 10007c80 f   Memorylib.obj
 0001:00006c88       __ehhandler$?MemPoolSnapshotDestroy@@YGXPAU_HMEMPOOLSHOT@@@Z 10007c88 f   Memorylib.obj
 0001:00006ca0       __unwindfunclet$?MemPoolUnlock@@YGXPAU_HMEMPOOL@@@Z$0 10007ca0 f   Memorylib.obj
 0001:00006ca8       __ehhandler$?MemPoolUnlock@@YGXPAU_HMEMPOOL@@@Z 10007ca8 f   Memorylib.obj
 0001:00006cc0       __unwindfunclet$?MemPoolValidate@@YGXPAU_HMEMPOOL@@@Z$0 10007cc0 f   Memorylib.obj
 0001:00006cc8       __ehhandler$?MemPoolValidate@@YGXPAU_HMEMPOOL@@@Z 10007cc8 f   Memorylib.obj
 0001:00006ce0       __unwindfunclet$?MemPoolWalkDestroy@@YGXPAU_HMEMPOOLWALK@@@Z$0 10007ce0 f   Memorylib.obj
 0001:00006ce8       __ehhandler$?MemPoolWalkDestroy@@YGXPAU_HMEMPOOLWALK@@@Z 10007ce8 f   Memorylib.obj
 0001:00006d00       __unwindfunclet$?MemPoolWalkFirst@@YGPAU_HMEMPOOLWALK@@PAU_HMEMPOOLSHOT@@AAUMEMBLOCKINFO@@@Z$0 10007d00 f   Memorylib.obj
 0001:00006d08       __ehhandler$?MemPoolWalkFirst@@YGPAU_HMEMPOOLWALK@@PAU_HMEMPOOLSHOT@@AAUMEMBLOCKINFO@@@Z 10007d08 f   Memorylib.obj
 0001:00006d20       __unwindfunclet$?MemPoolWalkNext@@YG_NPAU_HMEMPOOLWALK@@AAUMEMBLOCKINFO@@@Z$0 10007d20 f   Memorylib.obj
 0001:00006d28       __ehhandler$?MemPoolWalkNext@@YG_NPAU_HMEMPOOLWALK@@AAUMEMBLOCKINFO@@@Z 10007d28 f   Memorylib.obj
 0001:00006d40       __unwindfunclet$?MemSize@@YGXAAI0@Z$0 10007d40 f   Memorylib.obj
 0001:00006d48       __ehhandler$?MemSize@@YGXAAI0@Z 10007d48 f   Memorylib.obj
 0001:00006d60       __unwindfunclet$?MemStringAlloc@@YGPAXII@Z$0 10007d60 f   Memorylib.obj
 0001:00006d68       __ehhandler$?MemStringAlloc@@YGPAXII@Z 10007d68 f   Memorylib.obj
 0001:00006d80       __unwindfunclet$?MemStringFree@@YGXPAX@Z$0 10007d80 f   Memorylib.obj
 0001:00006d88       __ehhandler$?MemStringFree@@YGXPAX@Z 10007d88 f   Memorylib.obj
 0001:00006da0       __unwindfunclet$?MemVMDumpPool@@YGXPBD0@Z$0 10007da0 f   Memorylib.obj
 0001:00006da8       __ehhandler$?MemVMDumpPool@@YGXPBD0@Z 10007da8 f   Memorylib.obj
 0001:00006dc0       __unwindfunclet$?MemVMMap@@YGHPBD@Z$0 10007dc0 f   Memorylib.obj
 0001:00006dc8       __ehhandler$?MemVMMap@@YGHPBD@Z 10007dc8 f   Memorylib.obj
 0001:00006de0       __unwindfunclet$?MemoryManagerShutdown@@YGXXZ$0 10007de0 f   Memorylib.obj
 0001:00006de8       __ehhandler$?MemoryManagerShutdown@@YGXXZ 10007de8 f   Memorylib.obj
 0001:00006e00       __unwindfunclet$??1MemPoolSmall@@QAE@XZ$0 10007e00 f   MemorySmall.obj
 0001:00006e08       __ehhandler$??1MemPoolSmall@@QAE@XZ 10007e08 f   MemorySmall.obj
 0001:00006e20       __unwindfunclet$??1SmallInternals@?A0x79a48f2f@@AAE@XZ$0 10007e20 f   MemorySmall.obj
 0001:00006e28       __ehhandler$??1SmallInternals@?A0x79a48f2f@@AAE@XZ 10007e28 f   MemorySmall.obj
 0001:00006e40       __unwindfunclet$??4MemPoolSmall@@QAEAAV0@ABV0@@Z$1 10007e40 f   MemorySmall.obj
 0001:00006e48       __ehhandler$??4MemPoolSmall@@QAEAAV0@ABV0@@Z 10007e48 f   MemorySmall.obj
 0001:00006e60       __unwindfunclet$?Alloc@SmallInternals@?A0x79a48f2f@@QAEPAXI@Z$0 10007e60 f   MemorySmall.obj
 0001:00006e68       __ehhandler$?Alloc@SmallInternals@?A0x79a48f2f@@QAEPAXI@Z 10007e68 f   MemorySmall.obj
 0001:00006e80       __unwindfunclet$?Free@MemPoolSmall@@QAEXPAXI@Z$0 10007e80 f   MemorySmall.obj
 0001:00006e88       __ehhandler$?Free@MemPoolSmall@@QAEXPAXI@Z 10007e88 f   MemorySmall.obj
 0001:00006ea0       __unwindfunclet$?Free@SmallInternals@?A0x79a48f2f@@QAEXPAXI@Z$0 10007ea0 f   MemorySmall.obj
 0001:00006ea8       __ehhandler$?Free@SmallInternals@?A0x79a48f2f@@QAEXPAXI@Z 10007ea8 f   MemorySmall.obj
 0001:00006ec0       __unwindfunclet$?Release@SmallInternals@?A0x79a48f2f@@QAEXXZ$0 10007ec0 f   MemorySmall.obj
 0001:00006ec8       __ehhandler$?Release@SmallInternals@?A0x79a48f2f@@QAEXXZ 10007ec8 f   MemorySmall.obj
 0001:00006ee0       __unwindfunclet$?DumpMemRegions@@YG_NPAXPBD1@Z$0 10007ee0 f   mmPeek.obj
 0001:00006ee8       __unwindfunclet$?DumpMemRegions@@YG_NPAXPBD1@Z$1 10007ee8 f   mmPeek.obj
 0001:00006ef0       __ehhandler$?DumpMemRegions@@YG_NPAXPBD1@Z 10007ef0 f   mmPeek.obj
 0001:00006f00       __unwindfunclet$?DumpWorkingSet@@YG_NPAXPBD@Z$0 10007f00 f   mmPeek.obj
 0001:00006f08       __unwindfunclet$?DumpWorkingSet@@YG_NPAXPBD@Z$1 10007f08 f   mmPeek.obj
 0001:00006f10       __ehhandler$?DumpWorkingSet@@YG_NPAXPBD@Z 10007f10 f   mmPeek.obj
 0001:00006f20       __unwindfunclet$?Create@MMPoolVM@@SGPAV1@PBDI@Z$0 10007f20 f   mmPoolVM.obj
 0001:00006f31       __ehhandler$?Create@MMPoolVM@@SGPAV1@PBDI@Z 10007f31 f   mmPoolVM.obj
 0001:00006f40       __ehhandler$?_Copy@?$basic_string@DU?$char_traits@D@std@@V?$allocator@D@2@@std@@QAEXII@Z 10007f40 f   mmgr.obj
 0001:00006f50       ??__E?_Generic_object@?$_Error_objects@H@std@@2V_Generic_error_category@2@A@@YAXXZ 10007f50 f   mmgr.obj
 0001:00006f60       ??__E?_Iostream_object@?$_Error_objects@H@std@@2V_Iostream_error_category@2@A@@YAXXZ 10007f60 f   mmgr.obj
 0001:00006f70       ??__E?_System_object@?$_Error_objects@H@std@@2V_System_error_category@2@A@@YAXXZ 10007f70 f   mmgr.obj
 0001:00006f80       ??__F?_Generic_object@?$_Error_objects@H@std@@2V_Generic_error_category@2@A@@YAXXZ 10007f80 f   mmgr.obj
 0001:00006f90       ??__F?_Iostream_object@?$_Error_objects@H@std@@2V_Iostream_error_category@2@A@@YAXXZ 10007f90 f   mmgr.obj
 0001:00006fa0       ??__F?_System_object@?$_Error_objects@H@std@@2V_System_error_category@2@A@@YAXXZ 10007fa0 f   mmgr.obj
 0002:00000388       _AllocEntrySizePrimes      10008388     mmPool.obj
 0002:000007dc       _GS_ExceptionPointers      100087dc     MSVCRT:gs_report.obj
 0002:00000b88       __unwindtable$?MemPoolCreate@@YGPAU_HMEMPOOL@@PBDI@Z 10008b88     Memorylib.obj
 0002:00000b90       __ehfuncinfo$?MemPoolCreate@@YGPAU_HMEMPOOL@@PBDI@Z 10008b90     Memorylib.obj
 0002:00000bb4       __unwindtable$?MemPoolDestroy@@YGXPAU_HMEMPOOL@@@Z 10008bb4     Memorylib.obj
 0002:00000bbc       __ehfuncinfo$?MemPoolDestroy@@YGXPAU_HMEMPOOL@@@Z 10008bbc     Memorylib.obj
 0002:00000be0       __unwindtable$?MemPoolName@@YGPBDPAU_HMEMPOOL@@@Z 10008be0     Memorylib.obj
 0002:00000be8       __ehfuncinfo$?MemPoolName@@YGPBDPAU_HMEMPOOL@@@Z 10008be8     Memorylib.obj
 0002:00000c0c       __unwindtable$?MemPoolAlloc@@YGPAXPAU_HMEMPOOL@@I@Z 10008c0c     Memorylib.obj
 0002:00000c14       __ehfuncinfo$?MemPoolAlloc@@YGPAXPAU_HMEMPOOL@@I@Z 10008c14     Memorylib.obj
 0002:00000c38       __unwindtable$?MemPoolFree@@YGXPAU_HMEMPOOL@@PAX@Z 10008c38     Memorylib.obj
 0002:00000c40       __ehfuncinfo$?MemPoolFree@@YGXPAU_HMEMPOOL@@PAX@Z 10008c40     Memorylib.obj
 0002:00000c64       __unwindtable$?MemPoolLock@@YGXPAU_HMEMPOOL@@@Z 10008c64     Memorylib.obj
 0002:00000c6c       __ehfuncinfo$?MemPoolLock@@YGXPAU_HMEMPOOL@@@Z 10008c6c     Memorylib.obj
 0002:00000c90       __unwindtable$?MemPoolUnlock@@YGXPAU_HMEMPOOL@@@Z 10008c90     Memorylib.obj
 0002:00000c98       __ehfuncinfo$?MemPoolUnlock@@YGXPAU_HMEMPOOL@@@Z 10008c98     Memorylib.obj
 0002:00000cbc       __unwindtable$?MemPoolValidate@@YGXPAU_HMEMPOOL@@@Z 10008cbc     Memorylib.obj
 0002:00000cc4       __ehfuncinfo$?MemPoolValidate@@YGXPAU_HMEMPOOL@@@Z 10008cc4     Memorylib.obj
 0002:00000ce8       __unwindtable$?MemPoolSize@@YGXPAU_HMEMPOOL@@AAI1@Z 10008ce8     Memorylib.obj
 0002:00000cf0       __ehfuncinfo$?MemPoolSize@@YGXPAU_HMEMPOOL@@AAI1@Z 10008cf0     Memorylib.obj
 0002:00000d14       __unwindtable$?MemPoolSnapshot@@YGPAU_HMEMPOOLSHOT@@PAU_HMEMPOOL@@@Z 10008d14     Memorylib.obj
 0002:00000d1c       __ehfuncinfo$?MemPoolSnapshot@@YGPAU_HMEMPOOLSHOT@@PAU_HMEMPOOL@@@Z 10008d1c     Memorylib.obj
 0002:00000d40       __unwindtable$?MemPoolSnapshotDestroy@@YGXPAU_HMEMPOOLSHOT@@@Z 10008d40     Memorylib.obj
 0002:00000d48       __ehfuncinfo$?MemPoolSnapshotDestroy@@YGXPAU_HMEMPOOLSHOT@@@Z 10008d48     Memorylib.obj
 0002:00000d6c       __unwindtable$?MemPoolWalkFirst@@YGPAU_HMEMPOOLWALK@@PAU_HMEMPOOLSHOT@@AAUMEMBLOCKINFO@@@Z 10008d6c     Memorylib.obj
 0002:00000d74       __ehfuncinfo$?MemPoolWalkFirst@@YGPAU_HMEMPOOLWALK@@PAU_HMEMPOOLSHOT@@AAUMEMBLOCKINFO@@@Z 10008d74     Memorylib.obj
 0002:00000d98       __unwindtable$?MemPoolWalkNext@@YG_NPAU_HMEMPOOLWALK@@AAUMEMBLOCKINFO@@@Z 10008d98     Memorylib.obj
 0002:00000da0       __ehfuncinfo$?MemPoolWalkNext@@YG_NPAU_HMEMPOOLWALK@@AAUMEMBLOCKINFO@@@Z 10008da0     Memorylib.obj
 0002:00000dc4       __unwindtable$?MemPoolWalkDestroy@@YGXPAU_HMEMPOOLWALK@@@Z 10008dc4     Memorylib.obj
 0002:00000dcc       __ehfuncinfo$?MemPoolWalkDestroy@@YGXPAU_HMEMPOOLWALK@@@Z 10008dcc     Memorylib.obj
 0002:00000df0       __unwindtable$?MemSize@@YGXAAI0@Z 10008df0     Memorylib.obj
 0002:00000df8       __ehfuncinfo$?MemSize@@YGXAAI0@Z 10008df8     Memorylib.obj
 0002:00000e1c       __unwindtable$?MemVMMap@@YGHPBD@Z 10008e1c     Memorylib.obj
 0002:00000e24       __ehfuncinfo$?MemVMMap@@YGHPBD@Z 10008e24     Memorylib.obj
 0002:00000e48       __unwindtable$?MemVMDumpPool@@YGXPBD0@Z 10008e48     Memorylib.obj
 0002:00000e50       __ehfuncinfo$?MemVMDumpPool@@YGXPBD0@Z 10008e50     Memorylib.obj
 0002:00000e74       __unwindtable$?MemoryManagerShutdown@@YGXXZ 10008e74     Memorylib.obj
 0002:00000e7c       __ehfuncinfo$?MemoryManagerShutdown@@YGXXZ 10008e7c     Memorylib.obj
 0002:00000ea0       __unwindtable$?MemCRTAlloc@@YGPAXIH@Z 10008ea0     Memorylib.obj
 0002:00000ea8       __ehfuncinfo$?MemCRTAlloc@@YGPAXIH@Z 10008ea8     Memorylib.obj
 0002:00000ecc       __unwindtable$?MemCRTFree@@YGXPAXH@Z 10008ecc     Memorylib.obj
 0002:00000ed4       __ehfuncinfo$?MemCRTFree@@YGXPAXH@Z 10008ed4     Memorylib.obj
 0002:00000ef8       __unwindtable$?MemStringAlloc@@YGPAXII@Z 10008ef8     Memorylib.obj
 0002:00000f00       __ehfuncinfo$?MemStringAlloc@@YGPAXII@Z 10008f00     Memorylib.obj
 0002:00000f24       __unwindtable$?MemStringFree@@YGXPAX@Z 10008f24     Memorylib.obj
 0002:00000f2c       __ehfuncinfo$?MemStringFree@@YGXPAX@Z 10008f2c     Memorylib.obj
 0002:00000f50       __unwindtable$??1MemPoolSmall@@QAE@XZ 10008f50     MemorySmall.obj
 0002:00000f58       __ehfuncinfo$??1MemPoolSmall@@QAE@XZ 10008f58     MemorySmall.obj
 0002:00000f7c       __unwindtable$??4MemPoolSmall@@QAEAAV0@ABV0@@Z 10008f7c     MemorySmall.obj
 0002:00000f84       __ehfuncinfo$??4MemPoolSmall@@QAEAAV0@ABV0@@Z 10008f84     MemorySmall.obj
 0002:00000fa8       __unwindtable$?Free@MemPoolSmall@@QAEXPAXI@Z 10008fa8     MemorySmall.obj
 0002:00000fb0       __ehfuncinfo$?Free@MemPoolSmall@@QAEXPAXI@Z 10008fb0     MemorySmall.obj
 0002:00000fd4       __unwindtable$??1SmallInternals@?A0x79a48f2f@@AAE@XZ 10008fd4     MemorySmall.obj
 0002:00000fdc       __ehfuncinfo$??1SmallInternals@?A0x79a48f2f@@AAE@XZ 10008fdc     MemorySmall.obj
 0002:00001000       __unwindtable$?Release@SmallInternals@?A0x79a48f2f@@QAEXXZ 10009000     MemorySmall.obj
 0002:00001008       __ehfuncinfo$?Release@SmallInternals@?A0x79a48f2f@@QAEXXZ 10009008     MemorySmall.obj
 0002:0000102c       __unwindtable$?Alloc@SmallInternals@?A0x79a48f2f@@QAEPAXI@Z 1000902c     MemorySmall.obj
 0002:00001034       __ehfuncinfo$?Alloc@SmallInternals@?A0x79a48f2f@@QAEPAXI@Z 10009034     MemorySmall.obj
 0002:00001058       __unwindtable$?Free@SmallInternals@?A0x79a48f2f@@QAEXPAXI@Z 10009058     MemorySmall.obj
 0002:00001060       __ehfuncinfo$?Free@SmallInternals@?A0x79a48f2f@@QAEXPAXI@Z 10009060     MemorySmall.obj
 0002:00001084       __unwindtable$?DumpWorkingSet@@YG_NPAXPBD@Z 10009084     mmPeek.obj
 0002:00001094       __ehfuncinfo$?DumpWorkingSet@@YG_NPAXPBD@Z 10009094     mmPeek.obj
 0002:000010b8       __unwindtable$?DumpMemRegions@@YG_NPAXPBD1@Z 100090b8     mmPeek.obj
 0002:000010c8       __ehfuncinfo$?DumpMemRegions@@YG_NPAXPBD1@Z 100090c8     mmPeek.obj
 0002:000010ec       __unwindtable$?Create@MMPoolVM@@SGPAV1@PBDI@Z 100090ec     mmPoolVM.obj
 0002:000010f4       __ehfuncinfo$?Create@MMPoolVM@@SGPAV1@PBDI@Z 100090f4     mmPoolVM.obj
 0002:00001118       __catchsym$?_Copy@?$basic_string@DU?$char_traits@D@std@@V?$allocator@D@2@@std@@QAEXII@Z$5 10009118     mmgr.obj
 0002:00001128       __catchsym$?_Copy@?$basic_string@DU?$char_traits@D@std@@V?$allocator@D@2@@std@@QAEXII@Z$4 10009128     mmgr.obj
 0002:00001138       __unwindtable$?_Copy@?$basic_string@DU?$char_traits@D@std@@V?$allocator@D@2@@std@@QAEXII@Z 10009138     mmgr.obj
 0002:00001158       __ehfuncinfo$?_Copy@?$basic_string@DU?$char_traits@D@std@@V?$allocator@D@2@@std@@QAEXII@Z 10009158     mmgr.obj
 0002:0000117c       __tryblocktable$?_Copy@?$basic_string@DU?$char_traits@D@std@@V?$allocator@D@2@@std@@QAEXII@Z 1000917c     mmgr.obj
 0002:000011a8       __sehtable$__onexit        100091a8     MSVCRT:atonexit.obj
 0002:000011c8       __sehtable$??_M@YGXPAXIHP6EX0@Z@Z 100091c8     MSVCRT:ehvecdtr.obj
 0002:000011e8       __sehtable$?__ArrayUnwind@@YGXPAXIHP6EX0@Z@Z 100091e8     MSVCRT:ehvecdtr.obj
 0002:00001602       .idata$6                   10009602     kernel32:KERNEL32.dll
 0002:0000162a       .idata$6                   1000962a     user32:USER32.dll
 0002:000016d0       .idata$6                   100096d0     msvcprt:MSVCP110.dll
 0002:0000175e       .idata$6                   1000975e     MSVCRT:MSVCR110.dll
 0002:00001890       .edata                     10009890     Memory.exp
 0002:000018b8       rgpv                       100098b8     Memory.exp
 0002:00001990       rgszName                   10009990     Memory.exp
 0002:00001a68       rgwOrd                     10009a68     Memory.exp
 0002:00001ad4       szName                     10009ad4     Memory.exp
 0002:00001adf       $N00001                    10009adf     Memory.exp
 0002:00001afc       $N00002                    10009afc     Memory.exp
 0002:00001b17       $N00003                    10009b17     Memory.exp
 0002:00001b35       $N00004                    10009b35     Memory.exp
 0002:00001b52       $N00005                    10009b52     Memory.exp
 0002:00001b6a       $N00006                    10009b6a     Memory.exp
 0002:00001b83       $N00007                    10009b83     Memory.exp
 0002:00001ba4       $N00008                    10009ba4     Memory.exp
 0002:00001bc6       $N00009                    10009bc6     Memory.exp
 0002:00001be5       $N00010                    10009be5     Memory.exp
 0002:00001c04       $N00011                    10009c04     Memory.exp
 0002:00001c2f       $N00012                    10009c2f     Memory.exp
 0002:00001c50       $N00013                    10009c50     Memory.exp
 0002:00001c8a       $N00014                    10009c8a     Memory.exp
 0002:00001cc4       $N00015                    10009cc4     Memory.exp
 0002:00001cea       $N00016                    10009cea     Memory.exp
 0002:00001cff       $N00017                    10009cff     Memory.exp
 0002:00001d26       $N00018                    10009d26     Memory.exp
 0002:00001d4a       $N00019                    10009d4a     Memory.exp
 0002:00001d6f       $N00020                    10009d6f     Memory.exp
 0002:00001d94       $N00021                    10009d94     Memory.exp
 0002:00001db9       $N00022                    10009db9     Memory.exp
 0002:00001ddb       $N00023                    10009ddb     Memory.exp
 0002:00001dff       $N00024                    10009dff     Memory.exp
 0002:00001e25       $N00025                    10009e25     Memory.exp
 0002:00001e5c       $N00026                    10009e5c     Memory.exp
 0002:00001e8d       $N00027                    10009e8d     Memory.exp
 0002:00001eb1       $N00028                    10009eb1     Memory.exp
 0002:00001ed7       $N00029                    10009ed7     Memory.exp
 0002:00001f04       $N00030                    10009f04     Memory.exp
 0002:00001f51       $N00031                    10009f51     Memory.exp
 0002:00001f8d       $N00032                    10009f8d     Memory.exp
 0002:00001fae       $N00033                    10009fae     Memory.exp
 0002:00001fc2       $N00034                    10009fc2     Memory.exp
 0002:00001fdc       $N00035                    10009fdc     Memory.exp
 0002:00001ff0       $N00036                    10009ff0     Memory.exp
 0002:00002004       $N00037                    1000a004     Memory.exp
 0002:00002020       $N00038                    1000a020     Memory.exp
 0002:0000203a       $N00039                    1000a03a     Memory.exp
 0002:00002053       $N00040                    1000a053     Memory.exp
 0002:00002071       $N00041                    1000a071     Memory.exp
 0002:00002090       $N00042                    1000a090     Memory.exp
 0002:000020a9       $N00043                    1000a0a9     Memory.exp
 0002:000020c4       $N00044                    1000a0c4     Memory.exp
 0002:000020e3       $N00045                    1000a0e3     Memory.exp
 0002:000020fe       $N00046                    1000a0fe     Memory.exp
 0002:0000211d       $N00047                    1000a11d     Memory.exp
 0002:0000213a       $N00048                    1000a13a     Memory.exp
 0002:00002154       $N00049                    1000a154     Memory.exp
 0002:0000216a       $N00050                    1000a16a     Memory.exp
 0002:00002186       $N00051                    1000a186     Memory.exp
 0002:0000219f       $N00052                    1000a19f     Memory.exp
 0002:000021de       $N00053                    1000a1de     Memory.exp
 0002:000021f6       $N00054                    1000a1f6     Memory.exp
 0003:00000020       _s_unique                  1000b020     mmPool.obj
 0003:00000158       _s_pools                   1000b158     Memorylib.obj
 0003:0000015c       _s_default                 1000b15c     Memorylib.obj
 0003:00000160       _s_string                  1000b160     Memorylib.obj
 0003:00000168       _s_writeLeakFile           1000b168     Memorylib.obj
 0003:00000274       _s_MPeek                   1000b274     mmPeek.obj
 0003:00000278       _s_GetModuleFileNameEx     1000b278     mmPeek.obj
 0003:0000027c       _s_GetMappedFileName       1000b27c     mmPeek.obj
 0003:00000280       _s_EmptyWorkingSet         1000b280     mmPeek.obj
 0003:00000284       _s_QueryWorkingSet         1000b284     mmPeek.obj
 0003:00000294       _s_POOLHEAP                1000b294     mmPool.obj
 0003:00000298       _s_INFOHEAP                1000b298     mmPool.obj
 0003:0000029c       _s_traces                  1000b29c     mmPool.obj
 0003:000002b0       _g_GlobalLockBuf           1000b2b0     mmThreadLock.obj
 0003:000002c8       ?line@?1??mmFormatAllocation@@YGPBDABQAU_HMEMPOOL@@ABUMEMBLOCKINFO@@I@Z@4PADA 1000b2c8     mmWriteHeap.obj
 0003:000022cc       _allocator_arg             1000d2cc     pch.obj
 0003:000022cd       _piecewise_construct       1000d2cd     pch.obj
 0003:000022d0       _gs_dwAllocGran            1000d2d0     VMQuery.obj
 0003:000022d4       _allocator_arg             1000d2d4     mmgr.obj
 0003:000022d5       _piecewise_construct       1000d2d5     mmgr.obj
 0003:000022e0       _GS_ExceptionRecord        1000d2e0     MSVCRT:gs_report.obj
 0003:00002330       _GS_ContextRecord          1000d330     MSVCRT:gs_report.obj
 0003:000025fc       _DebuggerWasPresent        1000d5fc     MSVCRT:gs_report.obj
 0004:00000000       ?_Generic_object$initializer$@?$_Error_objects@H@std@@2P6AXXZA 1000e000     mmgr.obj
 0004:00000004       ?_Iostream_object$initializer$@?$_Error_objects@H@std@@2P6AXXZA 1000e004     mmgr.obj
 0004:00000008       ?_System_object$initializer$@?$_Error_objects@H@std@@2P6AXXZA 1000e008     mmgr.obj
 0004:0000000c       _pinit                     1000e00c     MSVCRT:cpu_disp.obj
 0004:00000010       _pinit                     1000e010     MSVCRT:atonexit.obj
 0005:000000a0       $R000000                   1000f0a0     Memory.res
 0005:00000468       $R0003C8                   1000f468     Memory.res
